:020000040800F2
:10000000A02600200D020008B52B0008E9230008F7
:10001000E9280008990C0008D15D000800000000E4
:10002000000000000000000000000000FD32000899
:10003000A115000800000000452D0008D136000879
:1000400027020008270200082702000827020008EC
:1000500027020008270200082702000827020008DC
:10006000270200082702000827020008E50D000803
:10007000190F0008270200082702000827020008BD
:1000800027020008270200082702000827020008AC
:100090002702000827020008270200081D17000891
:1000A000270200082702000827020008270200088C
:1000B00027020008270200089539000827020008D7
:1000C000270200082702000827020008270200086C
:1000D00027020008C157000827020008270200086D
:1000E000270200082702000827020008270200084C
:1000F000270200082702000827020008270200083C
:10010000270200082702000827020008270200082B
:10011000270200082702000827020008270200081B
:10012000270200082702000827020008270200080B
:1001300000F002F800F05AF80AA090E8000C82449F
:100140008344AAF10107DA4501D100F04FF8AFF27C
:10015000090EBAE80F0013F0010F18BFFB1A43F0A5
:100160000103184730730000507300000A444FF039
:10017000000C10F8013B13F0070408BF10F8014B06
:100180001D1108BF10F8015B641E05D010F8016B4B
:10019000641E01F8016BF9D113F0080F1EBF10F8AF
:1001A000014BAD1C0C1B09D16D1E58BF01F801CBD2
:1001B000FAD505E014F8016B01F8016B6D1EF9D555
:1001C0009142D6D37047000000230024002500266A
:1001D000103A28BF78C1FBD8520728BF30C148BFAA
:1001E0000B6070471FB51FBD10B510BD00F0DAF8E9
:1001F0001146FFF7F7FF05F0C5FF00F0F8F803B46C
:10020000FFF7F2FF03BC00F0FFF800000948804749
:1002100009480047FEE7FEE7FEE7FEE7FEE7FEE7E8
:10022000FEE7FEE7FEE7FEE704480549054A064B00
:1002300070470000F536000831010008A0200020BA
:10024000A0260020A0220020A022002040EA0103D6
:1002500010B59B070FD1042A0DD310C808C9121F6F
:100260009C42F8D020BA19BA884201D9012010BDA9
:100270004FF0FF3010BD1AB1D30703D0521C07E076
:10028000002010BD10F8013B11F8014B1B1B07D1DA
:1002900010F8013B11F8014B1B1B01D1921EF1D14B
:1002A000184610BD40EA0103024630B59B0710D145
:1002B0004FF0013400E008C208C91D1B9D4315EA38
:1002C000C41FF8D013F0FF0102F8011B0DD01B0A68
:1002D000F8E711F8013B002B02F8013B05D011F8BB
:1002E000013B002B02F8013BF3D130BD10B5203AA1
:1002F000C0F00B80B1E81850203AA0E81850B1E8DF
:100300001850A0E81850BFF4F5AF5FEA027C24BF94
:10031000B1E81850A0E8185044BF18C918C0BDE88B
:1003200010405FEA827C24BF51F8043B40F8043B54
:1003300008BF7047D20728BF31F8023B48BF11F809
:10034000012B28BF20F8023B48BF00F8012B704763
:100350004FF0000200B5134694469646203922BF5E
:10036000A0E80C50A0E80C50B1F12001BFF4F7AFA9
:10037000090728BFA0E80C5048BF0CC05DF804EB8B
:10038000890028BF40F8042B08BF704748BF20F8F9
:10039000022B11F0804F18BF00F8012B70477047F7
:1003A00070477047754600F02BF8AE460500694669
:1003B000534620F00700854618B020B5FFF734FFFC
:1003C000BDE820404FF000064FF000074FF0000856
:1003D0004FF0000B21F00701AC46ACE8C009ACE8D7
:1003E000C009ACE8C009ACE8C0098D46704710B53B
:1003F0000446AFF300802046BDE81040FFF7FFBE83
:10040000004870474020002001491820ABBEFEE79D
:10041000260002007047000070B504460D461148E2
:10042000844205D01048844202D01048844200D152
:1004300004E04FF497710EA005F00EFD0DB1012DF3
:1004400000D104E040F22F1109A005F005FD25B10F
:10045000A06840F00100A06003E0A06820F0010067
:10046000A06070BD0024014000280140003C014014
:100470004C69627261726965735C53544D333246E4
:100480003130785F5374645065726970685F44728C
:10049000697665725C7372635C73746D3332663156
:1004A00030785F6164632E630000000070B504461D
:1004B0000D461048844202D00F48844200D104E027
:1004C00040F247110DA005F0C7FC0DB1012D00D180
:1004D00004E04FF4A47109A005F0BEFC25B1A068AA
:1004E00040F48070A06003E0A06820F48070A060F9
:1004F00070BD000000240140003C01404C69627264
:1005000061726965735C53544D3332463130785FA4
:100510005374645065726970685F4472697665727D
:100520005C7372635C73746D3332663130785F6113
:1005300064632E630000000010B50446194884422D
:1005400005D01948844202D01848844200D103E003
:10055000B62117A005F080FC1248844208D1012181
:10056000401502F00DFD0021601502F009FD17E0B5
:100570000D48844208D10121001502F001FD00213F
:10058000201502F0FDFC0BE00848844208D101214F
:10059000C80302F0F5FC00214FF4004002F0F0FC2B
:1005A00010BD00000024014000280140003C014033
:1005B0004C69627261726965735C53544D333246A3
:1005C0003130785F5374645065726970685F44724B
:1005D000697665725C7372635C73746D3332663115
:1005E00030785F6164632E630000000070B50446DC
:1005F00000250C48844205D00B48844202D00B48A9
:10060000844200D104E04FF4D97109A005F024FC24
:10061000A06800F0040008B1012500E0002528468C
:1006200070BD00000024014000280140003C014052
:100630004C69627261726965735C53544D33324622
:100640003130785F5374645065726970685F4472CA
:10065000697665725C7372635C73746D3332663194
:1006600030785F6164632E630000000070B504465B
:1006700000250C48844205D00B48844202D00B4828
:10068000844200D104E04FF4C67109A005F0E4FBF8
:10069000A06800F0080008B1012500E00025284608
:1006A00070BD00000024014000280140003C0140D2
:1006B0004C69627261726965735C53544D333246A2
:1006C0003130785F5374645065726970685F44724A
:1006D000697665725C7372635C73746D3332663114
:1006E00030785F6164632E63000000002DE9F04103
:1006F00005460C46002600275D48854205D05D482A
:10070000854202D05C48854200D103E0DF215BA036
:1007100005F0A2FB206818B32068B0F5803F1FD019
:100720002068B0F5003F1BD02068B0F5403F17D0DF
:100730002068B0F5802F13D02068B0F5A02F0FD01F
:100740002068B0F5C02F0BD02068B0F5E02F07D09F
:100750002068B0F5002F03D02068B0F5102F00D12D
:1007600003E0E02145A005F077FB207910B1207966
:10077000012800D103E0E12140A005F06DFB607984
:1007800010B16079012800D103E0E2213BA005F01F
:1007900063FBA06888B3A068B0F5003F2DD0A068C7
:1007A000B0F5802F29D0A068B0F5C02F25D0A06863
:1007B000B0F5002F21D0A068B0F5202F1DD0A06883
:1007C000B0F5402F19D0A068B0F5602F15D0A06803
:1007D00098B1A068B0F5003F0FD0A068B0F5C02F69
:1007E0000BD0A068B0F5002F07D0A068B0F5202F7F
:1007F00003D0A068B0F5402F00D103E0E3211FA093
:1008000005F02AFBE06818B1E068B0F5006F00D190
:1008100003E0E42119A005F01FFB207C012803DB85
:10082000207C102800DC03E0E52114A005F014FB77
:100830006E68214806402179206840EA012006437D
:100840006E60AE681D480640D4E902100843617925
:1008500040EA41000643AE60EE6A26F47006207C52
:10086000401EC0B2074346EA0756EE62BDE8F0817B
:100870000024014000280140003C01404C696272A4
:1008800061726965735C53544D3332463130785F21
:100890005374645065726970685F447269766572FA
:1008A0005C7372635C73746D3332663130785F6190
:1008B00064632E6300000000FFFEF0FFFDF7F1FF10
:1008C0002DE9F04706460C46174698460025A946EE
:1008D0006048864205D06048864202D05F48864222
:1008E00000D104E040F252215DA005F0B5FA0CB34E
:1008F000012C1FD0022C1DD0032C1BD0042C19D08E
:10090000052C17D0062C15D0072C13D0082C11D08D
:10091000092C0FD00A2C0DD00B2C0BD00C2C09D08D
:100920000D2C07D00E2C05D00F2C03D0102C01D08D
:10093000112C00D104E040F2532149A005F08CFABB
:10094000012F02DB102F00DC04E04FF4157144A0EE
:1009500005F082FAB8F1000F14D0B8F1010F11D0F0
:10096000B8F1020F0ED0B8F1030F0BD0B8F1040F9D
:1009700008D0B8F1050F05D0B8F1060F02D0B8F1D4
:10098000070F00D104E040F2552135A005F064FACC
:10099000092C13DDF568A4F10A0000EB40010720E3
:1009A00000FA01F925EA0905A4F10A0000EB40006C
:1009B00008FA00F945EA0905F5600EE0356904EB2F
:1009C0004401072000FA01F925EA090504EB440077
:1009D00008FA00F945EA09053561072F11DA756B48
:1009E000781E00EB80011F2000FA01F925EA0905B5
:1009F000781E00EB800004FA00F945EA09057563EA
:100A000026E00D2F11DA356BF81F00EB80011F2057
:100A100000FA01F925EA0905F81F00EB800004FA45
:100A200000F945EA0905356312E0F56AA7F10D0002
:100A300000EB80011F2000FA01F925EA0905A7F162
:100A40000D0000EB800004FA00F945EA0905F562A3
:100A5000BDE8F0870024014000280140003C01402F
:100A60004C69627261726965735C53544D333246EE
:100A70003130785F5374645065726970685F447296
:100A8000697665725C7372635C73746D3332663160
:100A900030785F6164632E630000000010B5044687
:100AA0000948844205D00948844202D0084884425B
:100AB00000D104E04FF4BF7106A005F0CDF9A068A5
:100AC00040F00800A06010BD002401400028014053
:100AD000003C01404C69627261726965735C5354F9
:100AE0004D3332463130785F5374645065726970AB
:100AF000685F4472697665725C7372635C73746D6F
:100B00003332663130785F6164632E630000000029
:100B100070B504460D461148844205D01048844201
:100B200002D01048844200D104E04FF4E6710EA0D8
:100B300005F092F90DB1012D00D104E040F2CD1184
:100B400009A005F089F925B1A06840F4A000A060D3
:100B500003E0A06820F4A000A06070BD0024014064
:100B600000280140003C01404C6962726172696575
:100B7000735C53544D3332463130785F5374645054
:100B800065726970685F4472697665725C737263DE
:100B90005C73746D3332663130785F6164632E63E9
:100BA0000000000010B504460948844205D00948F9
:100BB000844202D00848844200D104E04FF4D2714C
:100BC00006A005F049F9A06840F00400A06010BD3F
:100BD0000024014000280140003C01404C69627241
:100BE00061726965735C53544D3332463130785FBE
:100BF0005374645065726970685F44726976657297
:100C00005C7372635C73746D3332663130785F612C
:100C100064632E630000000030B5024600201FE030
:100C200000EB8003104C04EB83031B7B934216D133
:100C300000EB800314F8233083B9012300EB800418
:100C4000094D05F8243000EB80032C4604EB8303A8
:100C5000996000EB800304EB8303596002E0401CC1
:100C60000D28DDD300BF30BD9800002070B50546CB
:100C70000C4607480560012006490870642C00D224
:100C80006424264631460520FFF7C6FF70BD0000EC
:100C9000200000201C00002000BFFEE72DE9F04FDF
:100CA00091B004460D4692469B4600213548CDE959
:100CB00006103548CDE90410DDE9060101F052FBCC
:100CC00006460F462046294605F046FA80468946E4
:100CD000DDE9040101F046FBCDE90A015046594621
:100CE00005F03AFACDE9080142464B46DDE9080134
:100CF00006F0DAF9CDE90E0132463B46DDE90A019C
:100D000006F0D2F9CDE90C01DDE90C23DDE90E0195
:100D100005F032FE1D4AC2E914011046416D006D16
:100D200032463B46CDE9000106F07EF842464B468E
:100D3000CDE9020106F0ACF9144AC2E9160100BF80
:100D40001046416D006D4FF02042114BCDE902017C
:100D500006F02EF804D200210E480C4AC2E9141005
:100D60000A49D1E9160100220B4BCDE9020106F038
:100D700059F903D20021054A9165D16511B0BDE84A
:100D8000F08F00000000244000006940C8030020EC
:100D90009999B93F0000F03F00C072402DE9F04141
:100DA00005460E4617460B4C072002F077FC01F073
:100DB00047FCA56265B12660676040F6B830A06068
:100DC0000020A061A0614FF47A710720FFF724FF93
:100DD000BDE8F081B004002010B50446204602F0C2
:100DE0004BFA10BD10B50024022000F0DBF872B6FB
:100DF0003F4800683F4908603F484049096830F86B
:100E000011003B490968081A394908603C48408884
:100E100039493A4A126831F81210401A39490860C3
:100E2000374841883448354A126820F8121033494F
:100E3000096830F811002E49096808442C490860F7
:100E40002E480068401C2D49086040F2E24190FBAA
:100E5000F1F201FB1200294908602B48D0F8B410C8
:100E6000C0F8B010224801682748C0F8B410D0F884
:100E7000AC002549C1F8A8000846D0F8AC102348BA
:100E8000234A126830F81200091A1F48C0F8AC1043
:100E90001B4801881D481E4A126820F812101A4883
:100EA000D0F8AC0019491A4A126831F812100144FE
:100EB0001548C0F8AC1016490968491C144A084680
:100EC0001160C91700EB11710911A0EB011111603C
:100ED00062B601F011FA0F4A03C201F0ADF90D4AF2
:100EE000C2E9020101F0DEF90A4AC2E9040110BDBB
:100EF0004C00002048000020F80D00203C0000209D
:100F00003800002054000020C8030020BC17002037
:100F100040000020E00D002010B5302000F006F861
:100F200001200149086010BDB001214210B50446FE
:100F300004F0704010B10948204008B904B104E041
:100F400040F20E2106A004F087FF04F0805010B19B
:100F50001248046001E01248446010BD0000F0EF48
:100F60004C69627261726965735C53544D333246E9
:100F70003130785F5374645065726970685F447291
:100F8000697665725C7372635C73746D333266315B
:100F900030785F646D612E6300000000040402403D
:100FA0000000024010B5044604F0704010B109483A
:100FB000204008B904B104E040F2AF2106A004F0DB
:100FC0004BFF04F0805010B11248046001E0124859
:100FD000446010BD0000F0EF4C6962726172696597
:100FE000735C53544D3332463130785F53746450E0
:100FF00065726970685F4472697665725C7372636A
:101000005C73746D3332663130785F646D612E636A
:1010100000000000040402400000024070B50446D5
:101020000D46244884422AD022481430844226D0D7
:1010300020482830844222D01E483C3084421ED0B2
:101040001C48503084421AD01A486430844216D06A
:1010500018487830844212D0174884420FD016487E
:10106000143084420BD014482830844207D01248F0
:101070003C30844203D010485030844200D104E018
:1010800040F229110DA004F0E7FE0DB1012D00D1B1
:1010900004E04FF4957109A004F0DEFE25B120684C
:1010A00040F00100206004E020684FF6FE71084027
:1010B000206070BD08000240080402404C69627262
:1010C00061726965735C53544D3332463130785FD9
:1010D0005374645065726970685F447269766572B2
:1010E0005C7372635C73746D3332663130785F6445
:1010F0006D612E630000000010B504466A4884420A
:101100002AD069481430844226D067482830844267
:1011100022D065483C3084421ED06348503084421F
:101120001AD061486430844216D05F4878308442D7
:1011300012D05E4884420FD05C48143084420BD0F9
:101140005A482830844207D058483C30844203D063
:1011500056485030844200D103E06F2154A004F07F
:101160007BFE20684FF6FE71084020600020206062
:101170006060A060E0604C48844208D14A4808386A
:10118000406840F00F004849083948608AE0464806
:101190001430844208D144480838406840F0F000D8
:1011A0004149083948607DE03F482830844208D1F1
:1011B0003D480838406840F470603B490839486051
:1011C00070E039483C30844208D1374808384068DC
:1011D00040F4704034490839486063E03248503088
:1011E000844208D130480838406840F470202E49C5
:1011F0000839486056E02C486430844208D12A48B7
:101200000838406840F4700027490839486049E0D0
:1012100025487830844208D123480838406840F097
:1012200070602149083948603CE02048844206D17A
:10123000001F006840F00F00211F086032E01B48CB
:101240001430844208D11948001F006840F0F000B3
:101250001649091F086025E014482830844208D147
:101260001248001F006840F470601049091F0860B0
:1012700018E00E483C30844208D10C48001F00683A
:1012800040F470400949091F08600BE007485030DE
:10129000844207D10548001F006840F470200349CC
:1012A000091F086010BD0000080002400804024049
:1012B0004C69627261726965735C53544D33324696
:1012C0003130785F5374645065726970685F44723E
:1012D000697665725C7372635C73746D3332663108
:1012E00030785F646D612E630000000070B50446C5
:1012F0000D461646274884422AD026481430844298
:1013000026D024482830844222D022483C308442CF
:101310001ED02048503084421AD01E486430844287
:1013200016D01C487830844212D01B4884420FD01B
:101330001948143084420BD017482830844207D013
:1013400015483C30844203D013485030844200D1C9
:1013500004E040F2491111A004F07EFD25F00E00DA
:1013600008B905B104E04FF4A5710CA004F074FDB8
:101370000EB1012E00D104E040F24B1107A004F0A1
:101380006BFD1EB120682843206002E02068A8435E
:10139000206070BD08000240080402404C6962727F
:1013A00061726965735C53544D3332463130785FF6
:1013B0005374645065726970685F447269766572CF
:1013C0005C7372635C73746D3332663130785F6462
:1013D0006D612E630000000070B505460C460026C6
:1013E0005E4885422AD05D481430854226D05B484D
:1013F0002830854222D059483C3085421ED057487B
:10140000503085421AD055486430854216D0534832
:101410007830854212D0524885420FD0504814305F
:1014200085420BD04E482830854207D04C483C308E
:10143000854203D04A485030854200D103E0CF2195
:1014400048A004F009FDA068102801D0A06800B9E8
:1014500003E0D02143A004F0FFFCE06820B1E06885
:10146000B0F5803F00D203E0D1213EA004F0F4FCAF
:101470002069402801D0206900B903E0D22139A0B9
:1014800004F0EAFC6069802801D0606900B903E0DB
:10149000D32134A004F0E0FCA06938B1A069B0F514
:1014A000807F03D0A069B0F5007F00D103E0D42194
:1014B0002CA004F0D1FCE06938B1E069B0F5806F90
:1014C00003D0E069B0F5006F00D103E0D52125A07D
:1014D00004F0C2FC206A202801D0206A00B903E091
:1014E000D62120A004F0B8FC606AB0F5405F09D0B6
:1014F000606AB0F5005F05D0606AB0F5805F01D02A
:10150000606A00B903E0D72116A004F0A5FCA06A28
:10151000B0F5804F01D0A06A00B903E0D82111A036
:1015200004F09AFC2E6847F6F0708643216AA068A2
:1015300008432169084361690843A1690843E169D7
:101540000843616A0843A16A084306432E60E068C5
:1015500068602068A8606068E86070BD08000240AC
:10156000080402404C69627261726965735C53548D
:101570004D3332463130785F537464506572697010
:10158000685F4472697665725C7372635C73746DD4
:101590003332663130785F646D612E630000000085
:1015A000704701E000BF00BF011EA0F10100F9D1AA
:1015B0007047000010B50446FF21044880F81C1154
:1015C00002210E20FFF728FB10BD0000C8030020F9
:1015D00001460888704770B504460D4629462046E6
:1015E00000F0F4FA70BD000070B505460B461446D5
:1015F0002E465B0806480444002206E004EB420045
:10160000FFF7E6FF26F81200521C9A42F6D370BD8F
:1016100000F0070810B50446E00AC402204600F0B6
:1016200059FA10BD2DE9F04F85B082460F46164697
:10163000002004903748029078080190F00A35495C
:1016400001EBC029C6F30A06B819C0F30A0008B1B5
:10165000012000E00020B91900EBD12BC6F34900AE
:1016600000900024A0462546039403A800F01BFB2D
:10167000039818B9049805B0BDE8F08F002544E040
:1016800000240BE04FF4006101FB059101EB4400E5
:10169000FFF79EFF204921F81400641CB4F5806F09
:1016A000F0D30DB9009800E0002004460DE03AF8B0
:1016B0001800194921F814000198401E019008B93A
:1016C00000BF05E0641C08F10108B4F5806FEED39B
:1016D00000BF00F0C9FA09EBC520FFF79BFF00240B
:1016E0000BE04FF4006202FB059202EB44000A4A51
:1016F00032F81410FFF76FFF641CB4F5806FF0D35D
:1017000000F05AFAFF2004906D1C5D45B8D3049890
:10171000B1E7000000F00708DC17002010B54FF417
:10172000807000F06FF860B1012006490860002069
:1017300005490880881500F009F84FF4807000F022
:1017400033F810BD800000202404004010B504468A
:10175000200D000508B904B103E0D42102A004F073
:101760007BFB1048046010BD4C6962726172696550
:10177000735C53544D3332463130785F5374645048
:1017800065726970685F4472697665725C737263D2
:101790005C73746D3332663130785F657874692EAE
:1017A000630000001404014010B50446200D00053C
:1017B00008B904B103E0FC2102A004F04DFB10487D
:1017C000046010BD4C69627261726965735C535448
:1017D0004D3332463130785F5374645065726970AE
:1017E000685F4472697665725C7372635C73746D72
:1017F0003332663130785F657874692E630000009B
:101800001404014070B5044600250026012C31D097
:10181000022C2FD0042C2DD0082C2BD0102C29D00A
:10182000202C27D0402C25D0802C23D0B4F5807FCD
:1018300020D0B4F5007F1DD0B4F5806F1AD0B4F578
:10184000006F17D0B4F5805F14D0B4F5005F11D0ED
:10185000B4F5804F0ED0B4F5004F0BD0B4F5803FF7
:1018600008D0B4F5003F05D0B4F5802F02D0B4F510
:10187000002F00D103E0E52108A004F0EDFA16489E
:10188000006800EA0406144814300068204010B1D3
:101890000EB1012500E00025284670BD4C6962723A
:1018A00061726965735C53544D3332463130785FF1
:1018B0005374645065726970685F447269766572CA
:1018C0005C7372635C73746D3332663130785F655C
:1018D0007874692E630000000004014070B504466E
:1018E0000025207910B12079042800D103E06A2175
:1018F00035A004F0B1FA6079082805D060790C2889
:1019000002D06079102800D103E06B212EA004F0F2
:10191000A3FA20686FF3130010B9206800B103E048
:101920006C2129A004F098FAA07910B1A0790128BF
:1019300000D103E06D2124A004F08EFA314DA0798E
:1019400090B3284600682168884329460860081D2E
:10195000006821688843291D0860207905442868AB
:1019600021680843286027480830006821688843B8
:10197000244908310860081D00682168884321490E
:101980000C310860607910280FD1081F00682168A9
:1019900008431C4908310860081D00682168084395
:1019A00018490C3108600EE007E0164D60790544D7
:1019B000286821680843286005E0207905442868E4
:1019C00021688843286070BD4C69627261726965E4
:1019D000735C53544D3332463130785F53746450E6
:1019E00065726970685F4472697665725C73726370
:1019F0005C73746D3332663130785F657874692E4C
:101A000063000000000401400021016001710C210D
:101A100041710021817170470148006870470000E2
:101A200080000020002001490860704780000020ED
:101A300070B5064600250D4CFF200D4908700520A5
:101A400084F835010020C4F8380108E028466D1CF0
:101A50000A2804DD64210A20FFF708F904E00120C8
:101A600000F044FF0028F1D100BF70BDC803002082
:101A70005800002010B5044624F0350008B904B120
:101A800004E040F2B65103A004F0E6F91048C46047
:101A900010BD00004C69627261726965735C5354D9
:101AA0004D3332463130785F5374645065726970DB
:101AB000685F4472697665725C7372635C73746D9F
:101AC0003332663130785F666C6173682E63000074
:101AD0000020024070B504460425B4F1006F03D322
:101AE0001448844200D204E040F2A71112A004F08E
:101AF000B3F94FF4302000F0C3F80546042D17D198
:101B00001C48006940F002001A4908610846446117
:101B1000006940F0400008614FF4302000F0B0F858
:101B200005461448006941F6FD71084011490861F5
:101B3000284670BDFFFF0F084C69627261726965CB
:101B4000735C53544D3332463130785F5374645074
:101B500065726970685F4472697665725C737263FE
:101B60005C73746D3332663130785F666C617368B4
:101B70002E6300000020024004200B49C96801F0D8
:101B8000010109B101200EE00749C96801F0040113
:101B900009B1022007E00449C96801F0100109B148
:101BA000032000E004207047002002400148006A42
:101BB00070470000002002400348006940F08000A8
:101BC00001490861704700000020024070B50446DA
:101BD0000D460426B4F1006F03D31248844200D2AC
:101BE00004E040F25E3110A004F036F94FF40050EA
:101BF00000F046F80646042E11D11A48006940F05C
:101C00000100184908612580F00200F039F8064605
:101C10001448006941F6FE710840124908613046D7
:101C200070BD0000FFFF0F084C6962726172696548
:101C3000735C53544D3332463130785F5374645083
:101C400065726970685F4472697665725C7372630D
:101C50005C73746D3332663130785F666C617368C3
:101C60002E630000002002400248034948600348F8
:101C7000486070472301674500200240AB89EFCDE3
:101C800000B502460423FFF777FF034603E0FFF7A2
:101C900073FF0346521E012B01D1002AF7D102B96E
:101CA0000523184600BD38B504463520FFF7E2FE8F
:101CB000FFF77CFF0090009800F0C000206038BD66
:101CC00070B505460C4600265DB1012D09D0022DE8
:101CD00007D0032D05D0042D03D0052D01D0062DEE
:101CE00000D104E040F2652121A004F0B5F8ECB188
:101CF000012C1BD0022C19D0032C17D0042C15D08A
:101D0000052C13D0062C11D0072C0FD0082C0DD089
:101D1000092C0BD00A2C09D00B2C07D00C2C05D089
:101D20000D2C03D00E2C01D00F2C00D104E040F27A
:101D300066210FA004F090F8A007010F0F2000FA11
:101D400001F61A48A11050F82100B0431749A2101B
:101D500041F822000846A11050F82100A107090F00
:101D600005FA01F108431149A21041F8220070BDA3
:101D70004C69627261726965735C53544D333246CB
:101D80003130785F5374645065726970685F447273
:101D9000697665725C7372635C73746D333266313D
:101DA00030785F6770696F2E6300000008000140A3
:101DB0002DE9F05F05460C464FF00009CA460026A3
:101DC0000027B046B3465948854211D0584885424D
:101DD0000ED0584885420BD05748854208D0574806
:101DE000854205D05648854202D05648854200D1EA
:101DF00003E0B22154A004F02FF8E078A0B1E0781D
:101E0000042811D0E07828280ED0E07848280BD09C
:101E1000E078142808D0E078102805D0E0781C2855
:101E200002D0E078182800D103E0B32146A004F0E6
:101E300013F8002010B9208800B103E0B42142A0BB
:101E400004F00AF8E07800F00F09E07800F01000E4
:101E500080B1A078012805D0A078022802D0A0780F
:101E6000032800D103E0BB2137A003F0F5FFA078E1
:101E700040EA0909207838B3D5F8008000261FE031
:101E8000012000FA06F7208800EA070ABA4516D1B1
:101E9000B7000F2000FA07FB28EA0B0809FA07F041
:101EA00040EA0808E078282803D10120B0406861A2
:101EB00005E0E078482802D10120B0402861761C76
:101EC000082EDDD3C5F800802088FF282BDDD5F84B
:101ED0000480002623E006F10800012101FA00F742
:101EE000208800EA070ABA4518D1B7000F2000FA87
:101EF00007FB28EA0B0809FA07F040EA0808E0782F
:101F0000282803D106F1080081406961E07848285B
:101F100004D106F10800012181402961761C082EB8
:101F2000D9D3C5F80480BDE8F09F00000008014047
:101F3000000C014000100140001401400018014055
:101F4000001C0140002001404C69627261726965A9
:101F5000735C53544D3332463130785F5374645060
:101F600065726970685F4472697665725C737263EA
:101F70005C73746D3332663130785F6770696F2ED1
:101F8000630000002DE9F04704460E460027B846DE
:101F90000025A946012C7DD0022C7BD0042C79D0C1
:101FA000082C77D0694884427FD06848203084422A
:101FB0007BD06748844278D065488030844274D0B2
:101FC0006448844271D0644884426ED0634884423D
:101FD0006BD06348844268D06248844265D0B4F5CF
:101FE000805F62D0B4F5EA1F5FD0B4F5EB1F5CD020
:101FF000B4F5004F59D05C48844256D0401C84420E
:1020000053D0801C844250D0001D84424DD056488D
:102010000F30844249D0B4F1201F46D04FEAF0304F
:10202000844242D0514884423FD0514884423CD0FF
:102030005048844239D05048844236D04F48844278
:1020400033D0B4F5011F30D04D4884422DD0401C10
:1020500084422AD0801C844227D0001D844224D090
:1020600047480F30844220D045481F3084421CD05E
:1020700043483F30844218D041487F30844214D0D6
:102080003F48FF30844210D03E4884420DD03E4845
:10209000844200E009E008D03C48844205D03C4836
:1020A000844202D03B48844200D104E040F22A211D
:1020B00039A003F0D1FE0EB1012E00D104E040F2B0
:1020C0002B2135A003F0C8FE04F00040B0F1004F12
:1020D00002D14048C56901E03E484568C4F3034960
:1020E000A7B204F44010B0F5401F08D125F0706588
:1020F0003848406820F070603649486013E004F4C6
:102100008010B0F5801F07D1032000FA09F825EAF6
:10211000080545F0706506E0600D000107FA00F063
:10212000854345F0706526B1600D010107FA01F0A5
:10213000054304F00040B0F1004F02D12548C561CD
:1021400001E024484560BDE8F0870000100014005D
:1021500040001600000118000002180000031800DB
:1021600000081A00000C1A000100200000013000D5
:102170000002300000043000001120000020200088
:102180000100008000020080000400800008008040
:1021900000100080002000804C69627261726965E5
:1021A000735C53544D3332463130785F537464500E
:1021B00065726970685F4472697665725C73726398
:1021C0005C73746D3332663130785F6770696F2E7F
:1021D000630000000000014000B500F0A3FD40B91D
:1021E00001200A4981F8DC0000210848C0F8E0100D
:1021F0000BE000F087FD20B90420044981F8DC00E1
:1022000003E00020014981F8DC0000BDC803002084
:1022100070B5084801F0F4FE05B2064801F062FF0F
:1022200006B2A81904B2002C01DA604204B22046BA
:1022300070BD00000004004070B51549D1F8A80039
:1022400004F08BFD04460D460022124B2046294621
:1022500004F0EAFD04460D4600220F4B20462946B5
:1022600004F08AFB04460D4600220C4B204629460A
:1022700004F082FB04460D460022094B2046294605
:1022800004F07AFB04460D462046294670BD000046
:10229000C80300200088A34000FEAF400000224099
:1022A0000000304070B51049088804F06DFD044608
:1022B0000D4600220D4B2046294604F0B5FD04468C
:1022C0000D4600220A4B2046294604F055FB0446E1
:1022D0000D460022074B2046294604F04DFB0446DC
:1022E0000D462046294670BD380000200088A340D6
:1022F00000FEAF400000224070B51549D1F8B4008F
:1023000004F02BFD04460D460022124B20462946C0
:1023100004F08AFD04460D4600220F4B2046294654
:1023200004F02AFB04460D4600220C4B20462946A9
:1023300004F022FB04460D460022094B20462946A4
:1023400004F01AFB04460D462046294670BD0000E5
:10235000C80300200088A34000FEAF400000624098
:10236000008893402DE9F04104460D462046294659
:1023700003F0F2FE06460F463046394600F002F8FA
:10238000BDE8F0812DE9F05F04460D4600221346BA
:102390002046294604F048FC02D10020014610E006
:1023A0001048D0E9168342462046294604F07CFEB8
:1023B00082468B460B49D1E914834246594604F0C4
:1023C000DBFA06460F46002213463046394604F033
:1023D00029FE03D830463946BDE8F09F002001466B
:1023E000FAE70000C803002000BFFEE700B593B085
:1023F0000121084600F0F2FC01214FF4017000F0C9
:1024000079FD0320ADF8340000208DF837008DF8F9
:1024100036000DA94348FFF7CBFC4348FEF76CFE9E
:102420004248029042480390002004900220059008
:1024300000200690802007904000089080000990BE
:1024400020200A9000020B9000200C9002A9364830
:10245000FEF7C2FF012202213348FEF747FF0121A8
:102460003148FEF7DBFD0B208DF8040000208DF8CD
:1024700005008DF8060001208DF8070001A800F086
:102480009BFB2A484C38FEF757F8002000F06CFC04
:1024900000200E9001208DF83C008DF83D004FF497
:1024A000602010900020119002208DF848000EA9A5
:1024B0001E484C38FEF71AF90623012200211B485A
:1024C0004C38FEF7FDF907230222012117484C384A
:1024D000FEF7F6F9012115484C38FDF79DFF13482A
:1024E0004C38FEF7DBFA00BF10484C38FEF7BEF858
:1024F0000028F9D10D484C38FEF754FB00BF0B48BB
:102500004C38FEF773F80028F9D1012107484C3800
:10251000FDF7CCFF012105484C38FEF7F9FA13B05E
:1025200000BD000000080140080002404C240140AA
:102530003800002000B50020FEF74EFC00BD000072
:1025400000B58BB00121102000F0D4FC4FF4E070F6
:10255000ADF8100048208DF8130004A93548FFF7A6
:1025600027FC02A8FFF750FA4FF480700290002079
:102570008DF80C0008208DF80D0001208DF80E005C
:1025800002A8FFF7ABF908210220FFF799FB1720FB
:102590008DF8040000208DF805008DF8060001205C
:1025A0008DF8070001A800F007FB01212248FFF782
:1025B000E9FC0121022000F057FC08A802F0E2FA31
:1025C0000020ADF820004FF6FF70ADF82400002089
:1025D000ADF82600ADF8220008A9184802F0FAF973
:1025E00000231A460321154801F076FC05A801F0E6
:1025F00029FF05A9114801F0C9FD05A801F022FF36
:102600000420ADF8140005A90C4801F0BFFD01211C
:102610000A4801F0D3F901221146084801F01CFFD5
:102620000021064801F0B0FF0121044801F0D6FA6C
:102630000BB000BD00100140000C1A000004004067
:1026400070B54FF48D75034C0020E060206100F000
:1026500077FE70BDB0040020F8B500BF18264FF417
:10266000965090FBF6F74FF404712F48FDF770FE7B
:102670000B202D4981F834014FF4C87008804FF4C5
:10268000167048804FF4487088806420C8800881A4
:102690007820488141F28830A1F84800A1F84A002A
:1026A0004FF4F07088810A20C87319200874012043
:1026B000487400211D481C4AC2E9141000221A481F
:1026C0008265C26580884FF47A7148430A2190FB85
:1026D000F1F0322190FBF1F11348C0F8E010012035
:1026E000114981F8C80012A11448FDF7DBFD202133
:1026F00012489838FDF72CFE6946002003F0B6FC1E
:102700000E4D9435002405E007FB04F06E3025F8EB
:102710001400641C182CF7DB00F0FEFC00F0E0FC59
:1027200008B903F087FBF8BDC80300200000F03FA4
:1027300054465F434C592D3230313100080500209A
:1027400000B585B00120ADF80C0048208DF80F00D1
:1027500003208DF80E0003A91D48FFF729FB1E205A
:102760008DF8100000208DF811008DF81200012066
:102770008DF8130004A800F01FFA0121042000F0D6
:1027800073FB4FF6FF70ADF804000020ADF80000B9
:10279000ADF80600ADF8020069460E4802F01AF9DD
:1027A0000F23002211460B4801F0A8FA012211461E
:1027B000084801F051FE0021064801F0E5FE012124
:1027C000044801F00BFA00F02FFD05B000BD000039
:1027D000001801400008004010B503480349086094
:1027E00000F018F810BD0000C8030020040000200D
:1027F000012004490860044908600449086004494C
:10280000086070478C81224280012142840121426C
:10281000848121421CB5012144F2010000F06AFBD1
:102820004FF48060ADF8000004208DF80300694685
:102830002048FFF7BDFA4FF40070ADF80000032008
:102840008DF8020018208DF8030069461948FFF73B
:10285000AFFA4FF416501849086000208880C880ED
:10286000088188810C204881144803F0A5F94FF4B1
:10287000E06000F00FFA0B208DF8040001208DF8C5
:1028800006008DF8070001A800F096F925208DF8C4
:10289000040001A800F090F9012240F225510748F8
:1028A00003F0E6F80121054802F0E6FF01200449A3
:1028B00008601CBD00080140B4030020003801403E
:1028C000B0012142704700000549D1F8A01060F323
:1028D000C711034AC2F8A0100249086070470000FF
:1028E000C80300209881224200BFFEE710B50446CD
:1028F000FFF772FC24B900F077FE4FF0FF3010BDF7
:10290000554890F8DD00012801D1801EF7E75248B4
:1029100090F8DC00A04202D16FF00100EFE700F078
:1029200001FA28B900F0EEF910B96FF00200E6E7FD
:10293000494890F81A01012801D1401FDFE7002023
:1029400046490860052C72D2DFE804F07203224980
:1029500010000121404880F8DE100021C0F8E4108A
:10296000D0F8E0003C49C1F8E00062E000213A48BC
:1029700080F8DE1080884FF47A7148430A2190FB7A
:10298000F1F0322190FBF1F13348C0F8E41050E04F
:10299000314800884FF47A7148430A2190FBF1F0E6
:1029A000322190FBF1F12C48C0F8E41000884FF47C
:1029B0007A7148430A2190FBF1F0322190FBF1F14A
:1029C0002548D0F8E000814204DD0021224880F84B
:1029D000DE1003E00121204880F8DE1029E01E48C7
:1029E00040884FF47A7148430A2190FBF1F032217C
:1029F00090FBF1F11848C0F8E41040884FF47A7168
:102A000048430A2190FBF1F0322190FBF1F112488A
:102A1000D0F8E000814204DD00210F4880F8DE108C
:102A200003E001210C4880F8DE1002E0FFE700BF60
:102A300000BF00BF084890F8DE000949086000BFE9
:102A40000023084A0A21012000F07CFD024981F898
:102A5000DF00002053E70000C803002084812242E9
:102A6000808122424D3200082DE9F041064600F0F7
:102A700059F90746344648480068484890F81A0112
:102A800018B14FF0FF30BDE8F081444890F8DD0008
:102A900010B16FF00100F6E7404890F91901A0422B
:102AA00002D16FF00200EEE700F03CF938B14FF4CC
:102AB0007A710120FEF7DAF86FF00300E3E7374898
:102AC000807B10B96FF00400DDE7344981F81841CC
:102AD0000846007C2044401E097C90FBF1F201FB7B
:102AE0001200441C2D48007CA04200D100BF0121EF
:102AF0002A4880F81A1190F91901A04204DA2748EF
:102B000090F91901251A06E02448007C0119234890
:102B100090F919010D1A0020214908601F4981F818
:102B20001841012C03D0084690F8190138B91B4808
:102B3000B0F84A00322148431A49086007E01748B4
:102B4000B0F84800684332214843164908601548E8
:102B50000068B0F5803F02DB4FF6FF7001E01148DE
:102B6000006881B20D48A0F81E1101200E490860CE
:102B70000A4890F91C01401C10B10C4800F074FD8B
:102B800000230B4A2821012000F0DCFC034981F8D6
:102B90001C01002077E7000014812342C8030020B5
:102BA000908122421000002094812242E4040020FF
:102BB000B5150008704700002DE9F04104460025D6
:102BC00000270F26E07810B1E078012800D103E05B
:102BD000752121A003F040F96078102800DA03E0A5
:102BE00076211DA003F038F9A078102800DA03E060
:102BF000772119A003F030F9E07800B3224800688B
:102C000000F4E060C0F5E060050AC5F10407EE409D
:102C1000607800FA07F5A078304005432D011B4885
:102C200022788554207800F01F0101208840217807
:102C30004911890001F1E021C1F8000109E0207883
:102C400000F01F010120884011492278521141F8FB
:102C50002200BDE8F08100004C6962726172696512
:102C6000735C53544D3332463130785F5374645043
:102C700065726970685F4472697665725C737263CD
:102C80005C6D6973632E63000CED00E000E400E00E
:102C900080E100E010B50446B4F5E06F0BD0B4F568
:102CA000C06F08D0B4F5A06F05D0B4F5806F02D026
:102CB000B4F5407F00D103E0632104A003F0CCF819
:102CC0000E4820430E49086010BD00004C69627236
:102CD00061726965735C53544D3332463130785FAD
:102CE0005374645065726970685F44726976657286
:102CF0005C7372635C6D6973632E63000000FA0598
:102D00000CED00E00448807B10B104480068704777
:102D100003480068FBE70000C80300200C81234241
:102D20000481234200200449897B11B103490868CA
:102D300001E0034908687047C80300200881234266
:102D400000812342704700000549D1F8A01060F3CC
:102D50008611034AC2F8A0100249086070470000BB
:102D6000C80300209C81224270B50446002544B16E
:102D7000B4F5804F05D0B4F5004F02D0B4F5404F04
:102D800000D104E040F2023104A003F065F81248DB
:102D9000456825F440452543456070BD4C69627225
:102DA00061726965735C53544D3332463130785FDC
:102DB0005374645065726970685F447269766572B5
:102DC0005C7372635C73746D3332663130785F723A
:102DD00063632E63000000000010024070B50446DB
:102DE0000D4640F2575024EA000008B904B104E04F
:102DF00040F22B410CA003F02FF80DB1012D00D1B2
:102E000004E040F22C4108A003F026F82DB115484B
:102E1000406920431349486104E012484069A043D7
:102E20001049486170BD00004C6962726172696549
:102E3000735C53544D3332463130785F5374645071
:102E400065726970685F4472697665725C737263FB
:102E50005C73746D3332663130785F7263632E63F6
:102E6000000000000010024070B504460D461048F6
:102E7000204008B904B104E040F269410DA002F01D
:102E8000EBFF0DB1012D00D104E040F26A4109A031
:102E900002F0E2FF2DB11648C06920431449C86111
:102EA00004E01348C069A0431149C86170BD000027
:102EB000003601814C69627261726965735C5354BA
:102EC0004D3332463130785F5374645065726970A7
:102ED000685F4472697665725C7372635C73746D6B
:102EE0003332663130785F7263632E630000000016
:102EF0000010024070B504460D461048204008B945
:102F000004B104E040F24A410DA002F0A5FF0DB16A
:102F1000012D00D104E040F24B4109A002F09CFFDA
:102F20002DB11648806920431449886104E0134894
:102F30008069A0431149886170BD00000200C0FF94
:102F40004C69627261726965735C53544D333246E9
:102F50003130785F5374645065726970685F447291
:102F6000697665725C7372635C73746D333266315B
:102F700030785F7263632E6300000000001002402F
:102F800070B504460D461048204008B904B104E06D
:102F900040F2A4410DA002F05FFF0DB1012D00D160
:102FA00004E040F2A54109A002F056FF2DB11648F9
:102FB000C06820431449C86004E01348C068A043B7
:102FC0001149C86070BD00000200C0FF4C69627208
:102FD00061726965735C53544D3332463130785FAA
:102FE0005374645065726970685F44726976657283
:102FF0005C7372635C73746D3332663130785F7208
:1030000063632E63000000000010024030B5002111
:103010000022002400232D4D6D6805F00C0121B124
:10302000042905D0082923D105E0294D056022E0B7
:10303000274D05601FE0254D6D6805F47012234D86
:103040006D6805F48034022505EB92421CB9214DD0
:10305000554305600BE01D4D6D6805F400351DB14D
:103060001C4D5543056002E0194D5543056002E0D3
:10307000174D056000BF00BF144D6D6805F0F001ED
:103080000909154D6B5C0568DD4045600F4D6D68A5
:1030900005F4E061090A104D6B5C4568DD40856010
:1030A0000A4D6D6805F46051C90A0B4D6B5C4568AB
:1030B000DD40C560054D6D6805F44041890B074D45
:1030C0006B5CC568B5FBF3F5056130BD00100240CF
:1030D00000127A0000093D008400002094000020C6
:1030E00030B595B00024102250216846FEF77CFAD6
:1030F0004E21684602F072FF0546BDF84E00A84218
:1031000005D1502269460348FDF7F0F8641E2046B9
:1031100015B030BD180400200CB500220621684609
:10312000FEF762FABDF80000552805D1BDF802008F
:10313000044981F8340103E0FF20024981F8340199
:103140000CBD0000C80300202DE9FC4F00200090BA
:10315000314890F803B0D84645792846E91705EB81
:103160005171CC10E91705EB5171C910A5EBC101E4
:1031700009B1601CC4B200272CE0F81CC6B20020C4
:103180002649885582461BE001A9404602F0B2FF5D
:103190002248805D9DF8041001FA0AF108431F4996
:1031A000885508F1010000F0FF080BEB05004045D1
:1031B00002DC0120009006E00AF1010000F0FF0AA5
:1031C000BAF1080FE0DB00BF0098012800D103E04E
:1031D000781CC7B2A742D0DB00BF114890F8340179
:1031E0000E4908700220487008468470E01CC4B282
:1031F00021460A4802F0F2FE81464FEA292007499B
:103200000855601CC4B201F80490601C05490870A0
:1032100002F026FEBDE8FC8FB4020020B4010020BD
:10322000C80300200800002000210648C0F8D8107C
:10323000C0F8D41000200449086000210148C0F8FB
:10324000CC107047C80300202C00002010B50446A5
:10325000012007490860FF21064880F8DF1001219E
:1032600080F8DD1032210820FDF7D6FC10BD0000EB
:1032700084812242C803002030B50246114609B9B4
:1032800041F4805100241A4D2C60002001E000BF61
:10329000401C1028FBDB00231EE00124154D2C6090
:1032A00001F40044B4F5004F03D10124124D2C6009
:1032B00002E00024104D2C60002001E000BF401C03
:1032C0000E28FBDB00240B4D2C604900002000E0A1
:1032D000401C1028FCDB5B1C102BDEDB002001E017
:1032E00000BF401C0228FBDB0124014D2C6030BDD7
:1032F00090012142940121429C012142704700002B
:103300001CB50446074903C9CDE90001ADF80240E8
:10331000002206216846FEF785F9034880F834410B
:103320001CBD00007C740008C803002010B50122F9
:1033300040F22771014802F09BFB10BD00380140AC
:1033400070B50546124890F90000401C10B11048B5
:1033500000F08AF94FF47A706843FF2190FBF1F096
:103360000A2190FBF1F4002C0DDD002009490860D2
:10337000FF2D0BD00023084A2146012000F0E2F87F
:103380000349087002E001200249086070BD000096
:1033900034000020848121421136000810B500F06D
:1033A00001F810BD0CB50020019000903348006872
:1033B00040F480303149086000BF3048006800F4B4
:1033C000003000900198401C0190009818B90198B5
:1033D000B0F5A06FF1D12948006800F4003010B1B9
:1033E0000120009001E0002000900098012843D1C6
:1033F0002348006840F01000214908600846006832
:1034000020F0030008600846006840F002000860F1
:103410001A484068194948600846406848600846AC
:10342000406840F4806048600846406820F47C10A2
:1034300048600846406840F4A810486008460068A4
:1034400040F08070086000BF0C48006800F0007019
:103450000028F9D00948406820F003000749486077
:103460000846406840F00200486000BF03484068DA
:1034700000F00C000828F9D10CBD0000001002403B
:10348000002002402DE9F0410446204603F065FC8F
:10349000054602F061FE074688463846414600F080
:1034A00003F8BDE8F08100002DE9F04704460D4621
:1034B0000120224981F8C8000022214B20462946DC
:1034C00003F0B0FD01D200241D4D0022134620461A
:1034D000294603F06DFC01D2002425461749B1F8B6
:1034E000CA0003F051FC064622462B4603F09CFB23
:1034F0000AD020462946FEF745FF064603F0D0FBDA
:1035000082465046FDF768FC2046294603F0F8FB4A
:1035100081B20A48A0F8CA100146D1F8CC0003F0E5
:1035200033FC064622462B4603F072F9804603F030
:10353000E7FB0249C1F8CC00BDE8F087C8030020D2
:1035400000FEAF4070B504460D46164611490022F4
:103550001BE00878B0B924B1012C03D0022C03D1B0
:1035600001E000BF00BF03E000200870401E70BDF6
:1035700000BF4D608D60CE604C70012008700B6103
:1035800050B2F4E7501CC2B21431052AE1DB4FF00F
:10359000FF30ECE7DC1F0020002007E0002100EBFB
:1035A0008002044B03F82210411CC8B20528F5DB49
:1035B00070470000DC1F002000B500F001F800BDDE
:1035C00000B5084890F8C80050B10020054981F8BE
:1035D000C80000210348A0F8CA100020FDF7FCFB3A
:1035E00000BD0000C803002010B500200649086097
:1035F000064800F039F8082000F050F80021034890
:10360000DF3880F8DD1010BD84812242A70400203D
:103610000121034A1160FF21024A11707047000026
:10362000848121423400002010B500200449086044
:103630000021044880F81A110E2000F02FF810BD68
:1036400094812242C803002010B50020044908607C
:103650000021044880F81A110B2000F01FF810BD5B
:1036600094812242C8030020014691F900000528F8
:1036700003DA91F90000401C10B94FF0FF30704799
:10368000002091F9002002EB8202034B03F8220094
:10369000FF2008700020F2E7DC1F002010B5014673
:1036A00000200FE000EB8002084B03EB8202127B4C
:1036B0008A4206D1002200EB8003044C04F8232048
:1036C00002E0401C0D28EDD300BF10BD9800002083
:1036D00006480078012804D105480078401C0449B8
:1036E0000870012001490870704700009C0100200B
:1036F0009D01002010B51348006840F001001149F9
:10370000086008464068104908400E49486008466D
:1037100000680E4908400B4908600846006820F41C
:10372000802008600846406820F4FE0048604FF49E
:103730001F008860FFF732FE4FF000600449086008
:1037400010BD0000001002400000FFF8FFFFF6FE71
:1037500008ED00E0F0B50C46154600220021068C6D
:103760004FF6FE773E400684028B018C4FF60C76B6
:1037700032407E1C06EA03162E433243104EB042FE
:103780000ED0104EB0420BD0B0F1804F08D00E4E8C
:10379000B04205D00D4EB04202D00D4EB04206D11F
:1037A0004FF6FD76314044F00106314305E04FF617
:1037B000F576314044F00106314302830184F0BDC7
:1037C000002C01400034014000040040000800408B
:1037D000000C0040F0B50C461546002200210026E2
:1037E000078C4FF6EF7C07EA0C070784028B018CED
:1037F0004FF6FF7707EA041640F6FF473A404FF6C8
:10380000FF7707EA03373A434FF6FF7707EA0527C2
:103810003A43114FB8420ED0104FB8420BD0B0F11E
:10382000804F08D00E4FB84205D00E4FB84202D09C
:103830000D4FB84206D14FF6DF77394046F01007FA
:10384000394305E04FF65F77394044F010073943BC
:1038500002830184F0BD0000002C014000340140CF
:103860000004004000080040000C0040F0B50C4689
:103870001546002200210026078C4FF6FF6C07EA50
:103880000C070784828B018C4FF6FF7707EA04262A
:103890004FF60C773A404FF6FF7707EA03172F43AE
:1038A0003A43114FB8420ED0104FB8420BD0B0F18E
:1038B000804F08D00E4FB84205D00E4FB84202D00C
:1038C0000D4FB84206D14FF6FF57394046F4807786
:1038D000394305E04FF2FF57394044F480773943CC
:1038E00082830184F0BD0000002C014000340140BF
:1038F0000004004000080040000C0040F0B50C46F9
:103900001546002200210026078C4EF6FF7C07EAB0
:103910000C070784828B018C4FF6FF7707EA043689
:1039200040F6FF473A404FF6FF7707EA05273A434C
:103930004FF6FF7707EA03373A43114FB8420ED0EC
:10394000104FB8420BD0B0F1804F08D00E4FB842A4
:1039500005D00E4FB84202D00D4FB84206D14DF6F9
:10396000FF77394046F48057394305E047F6FF5763
:10397000394044F48057394382830184F0BD00000C
:10398000002C0140003401400004004000080040C9
:10399000000C004010B50648848C0121054800F059
:1039A00095F805480068401C0349086010BD0000F8
:1039B00000080040000800402C00002070B50446BC
:1039C0000D46234884422FD0B4F1804F2CD021489B
:1039D000844229D02048844226D02048844223D0E3
:1039E0001F48844220D01F4884421DD01E48844274
:1039F0001AD01E48844217D01D48844214D01D4856
:103A0000844211D01C4884420ED01C4884420BD002
:103A10001B48844208D01B48844205D01A4884427F
:103A200002D01A48844200D104E040F62B2118A0AD
:103A300002F012FA05F4614008B905B104E040F65D
:103A40002C2113A002F008FAE843208270BD000088
:103A5000002C01400004004000080040000C004021
:103A6000001000400014004000340140004C0140B0
:103A7000005001400054014000180040001C00406C
:103A80000020004000400140004401400048014047
:103A90004C69627261726965735C53544D3332468E
:103AA0003130785F5374645065726970685F447236
:103AB000697665725C7372635C73746D3332663100
:103AC00030785F74696D2E630000000070B50446A5
:103AD0000D46234884422FD0B4F1804F2CD021488A
:103AE000844229D02048844226D02048844223D0D2
:103AF0001F48844220D01F4884421DD01E48844263
:103B00001AD01E48844217D01D48844214D01D4844
:103B1000844211D01C4884420ED01C4884420BD0F1
:103B20001B48844208D01B48844205D01A4884426E
:103B300002D01A48844200D104E040F6772118A050
:103B400002F08AF905F47F4008B905B104E040F6B7
:103B5000782113A002F080F9E843208270BD0000B4
:103B6000002C01400004004000080040000C004010
:103B7000001000400014004000340140004C01409F
:103B8000005001400054014000180040001C00405B
:103B90000020004000400140004401400048014036
:103BA0004C69627261726965735C53544D3332467D
:103BB0003130785F5374645065726970685F447225
:103BC000697665725C7372635C73746D33326631EF
:103BD00030785F74696D2E630000000070B5044694
:103BE0000D46274884422FD0B4F1804F2CD0254871
:103BF000844229D02448844226D02448844223D0B9
:103C00002348844220D0234884421DD02248844245
:103C10001AD02248844217D02148844214D0214827
:103C2000844211D0204884420ED0204884420BD0D8
:103C30001F48844208D01F48844205D01E48844251
:103C400002D01E48844200D104E040F229311CA079
:103C500002F002F90DB1012D00D104E040F22A3149
:103C600017A002F0F9F825B1208840F0010020806B
:103C700004E020884FF6FE710840208070BD0000EF
:103C8000002C01400004004000080040000C0040EF
:103C9000001000400014004000340140004C01407E
:103CA000005001400054014000180040001C00403A
:103CB0000020004000400140004401400048014015
:103CC0004C69627261726965735C53544D3332465C
:103CD0003130785F5374645065726970685F447204
:103CE000697665725C7372635C73746D33326631CE
:103CF00030785F74696D2E63000000002DE9F0419B
:103D000004460D4616461F46224884420ED0B4F1A2
:103D1000804F0BD02048844208D02048844205D0F0
:103D20001F48844202D01F48844200D104E040F280
:103D300061411DA002F090F845B1B5F5805F05D056
:103D4000B5F5005F02D0B5F5405F00D104E040F268
:103D5000624115A002F080F8B6F5004F00D006B918
:103D600004E040F2634110A002F076F80F2F00DC6F
:103D700004E040F264410CA002F06EF83B4632468B
:103D80002946204600F02EF8208940F4804020810A
:103D9000BDE8F081002C0140000400400008004014
:103DA000000C0040003401404C6962726172696528
:103DB000735C53544D3332463130785F53746450E2
:103DC00065726970685F4472697665725C7372636C
:103DD0005C73746D3332663130785F74696D2E6355
:103DE000000000002DE9F04104460D4616461F462E
:103DF0004FF00008244884420ED0B4F1804F0BD01D
:103E00002248844208D02248844205D02148844276
:103E100002D02148844200D104E040F281411FA039
:103E200002F01AF845B1B5F5805F05D0B5F5005F31
:103E300002D0B5F5405F00D104E040F2824117A006
:103E400002F00AF8B6F5004F00D006B904E040F2DF
:103E5000834112A002F000F80F2F00DC04E040F2D2
:103E600084410EA001F0F8FFB4F8088008F0FF08C4
:103E70004FF6FF7000EA07203043284340EA080865
:103E8000A4F80880BDE8F081002C01400004004047
:103E900000080040000C0040003401404C69627290
:103EA00061726965735C53544D3332463130785FCB
:103EB0005374645065726970685F447269766572A4
:103EC0005C7372635C73746D3332663130785F7427
:103ED000696D2E63000000002DE9F04704460D4691
:103EE00016461F464FF00008C146C2462F4884427E
:103EF00011D0B4F1804F0ED02D4884420BD02D4804
:103F0000844208D02C48844205D02C48844202D0F8
:103F10002B48844200D104E04FF49F6129A001F0B6
:103F20009BFF012D03D0022D01D0032D00D104E011
:103F300040F2F94123A001F08FFF0EB1022E00D113
:103F400004E040F2FA411FA001F086FF0FB1022FFA
:103F500000D104E040F2FB411AA001F07DFFB4F86B
:103F60000880B4F81890B4F820A04FF6F87008EA6A
:103F7000000848EA05084FF6FC4009EA000940F24B
:103F8000011049EA00094FF6DD700AEA000A4FF60F
:103F9000FF7000EA0710304340EA0A0AA4F80880DC
:103FA000A4F81890A4F820A0BDE8F087002C0140E8
:103FB0000004004000080040000C004000340140B4
:103FC000004001404C69627261726965735C5354D0
:103FD0004D3332463130785F537464506572697086
:103FE000685F4472697665725C7372635C73746D4A
:103FF0003332663130785F74696D2E6300000000E3
:1040000010B504461A48844229D0B4F1804F26D016
:104010001848844223D01848844220D0174884424C
:104020001DD0174884421AD01648844217D016482B
:10403000844214D01548844211D0154884420ED0D1
:10404000144884420BD01448844208D01348844258
:1040500005D01348844202D01248844200D104E0C3
:1040600040F69C1110A001F0F7FEA08E10BD0000DC
:10407000002C01400004004000080040000C0040FB
:1040800000340140004C0140005001400054014008
:1040900000180040001C004000200040004001408B
:1040A00000440140004801404C69627261726965D8
:1040B000735C53544D3332463130785F53746450DF
:1040C00065726970685F4472697665725C73726369
:1040D0005C73746D3332663130785F74696D2E6352
:1040E0000000000010B504461148844217D0B4F116
:1040F000804F14D00F48844211D00F4884420ED014
:104100000E4884420BD00E48844208D00D488442A9
:1041100005D00D48844202D00C48844200D104E00E
:1041200040F6A9110AA001F097FE208F10BD0000F3
:10413000002C01400004004000080040000C00403A
:1041400000340140004C0140001800400040014094
:104150004C69627261726965735C53544D333246C7
:104160003130785F5374645065726970685F44726F
:10417000697665725C7372635C73746D3332663139
:1041800030785F74696D2E630000000070B50446DE
:104190000D46288840B12888042805D0288808289A
:1041A00002D028880C2800D104E040F24E2188A0DB
:1041B00001F052FEA888012805D0A888022802D064
:1041C000A888032800D104E040F24F2180A001F02C
:1041D00043FEE88840B1E888042805D0E88808282C
:1041E00002D0E8880C2800D104E04FF4147178A0C4
:1041F00001F032FE28890F2800DC04E040F2512152
:1042000073A001F029FE814884420ED08048844288
:104210000BD0B4F1804F08D07E48844205D07E4850
:10422000844202D07D4884420BD1688810B16888EE
:10423000022800D113E040F2562165A001F00CFEE7
:104240000DE0688828B16888022802D068880A28AA
:1042500000D104E040F25A215DA001F0FDFD288864
:1042600000283DD16948844229D0B4F1804F26D03E
:104270006848844223D06848844220D067488442FA
:104280001DD0634884421AD06548844217D06548DF
:10429000844214D06448844211D0644884420ED0D1
:1042A000634884420BD06348844208D06248844209
:1042B00005D06248844202D06148844200D104E0C3
:1042C00040F25E2142A001F0C7FD2B89AA886988CF
:1042D0002046FFF73FFAE988204600F0D1F976E062
:1042E000288804282BD14948844217D0B4F1804F44
:1042F00014D04848844211D0474884420ED04748E1
:1043000084420BD04248844208D04548844205D0BC
:104310004648844202D04848844200D104E04FF429
:104320001A712BA001F098FD2B89AA886988204674
:10433000FFF750FAE988204600F028FA47E028887D
:10434000082822D1314884420ED0B4F1804F0BD0DE
:104350003048844208D03048844205D02F488442F7
:1043600002D02B48844200D104E040F2722118A010
:1043700001F072FD2B89AA8869882046FFF776FA3A
:10438000E988204600F06EFA21E0204884420ED0F1
:10439000B4F1804F0BD01F48844208D01E4884429D
:1043A00005D01E48844202D01948844200D104E05E
:1043B0004FF41F7106A001F04FFD2B89AA88698870
:1043C0002046FFF79BFAE988204600F0A5FA70BD69
:1043D0004C69627261726965735C53544D33324645
:1043E0003130785F5374645065726970685F4472ED
:1043F000697665725C7372635C73746D33326631B7
:1044000030785F74696D2E6300000000002C01405D
:10441000003401400004004000080040000C00404F
:10442000004C014000500140005401400018004081
:10443000001C0040002000400040014000440140BA
:10444000004801400021018041800121818000213C
:10445000C18001817047000070B504460D461646C4
:104460002A4884422FD0B4F1804F2CD0284884426F
:1044700029D02848844226D02748844223D0274880
:10448000844220D0264884421DD0264884421AD037
:104490002548844217D02548844214D024488442B9
:1044A00011D0244884420ED0234884420BD02348A4
:1044B000844208D02248844205D02248844202D057
:1044C0002148844200D104E040F26B311FA001F08A
:1044D000C3FC05F47F4008B905B104E04FF45B71FB
:1044E0001AA001F0B9FC0EB1012E00D104E040F297
:1044F0006D3116A001F0B0FC1EB1A0892843A08147
:1045000002E0A089A843A08170BD0000002C0140FA
:104510000004004000080040000C00400010004073
:104520000014004000340140004C014000500140A4
:104530000054014000180040001C004000200040D2
:104540000040014000440140004801404C69627253
:1045500061726965735C53544D3332463130785F14
:104560005374645065726970685F447269766572ED
:104570005C7372635C73746D3332663130785F7470
:10458000696D2E630000000070B504460D461D489D
:1045900084422FD0B4F1804F2CD01B48844229D0C4
:1045A0001A48844226D01A48844223D019488442AB
:1045B00020D0194884421DD0184884421AD0184887
:1045C000844217D01748844214D01748844211D02F
:1045D000164884420ED0164884420BD015488442B7
:1045E00008D01548844205D01448844202D01448AB
:1045F000844200D104E040F6DB0112A001F02CFC63
:10460000A58470BD002C014000040040000800405B
:10461000000C004000100040001400400034014035
:10462000004C01400050014000540140001800407F
:10463000001C0040002000400040014000440140B8
:10464000004801404C69627261726965735C535441
:104650004D3332463130785F5374645065726970FF
:10466000685F4472697665725C7372635C73746DC3
:104670003332663130785F74696D2E63000000005C
:1046800070B504460D462448844229D0B4F1804FC9
:1046900026D02248844223D02148844220D0214879
:1046A00084421DD0204884421AD02048844217D02A
:1046B0001F48844214D01F48844211D01E488442AF
:1046C0000ED01E4884420BD01D48844208D01D489D
:1046D000844205D01C48844202D01C48844200D148
:1046E00004E040F634111AA001F0B6FB2DB1042D00
:1046F00003D0082D01D00C2D00D104E040F6351177
:1047000013A001F0A9FB208B4FF6F3710840208322
:10471000208B2843208370BD002C01400004004002
:1047200000080040000C004000340140004C0140F3
:10473000005001400054014000180040001C00409F
:10474000002000400040014000440140004801407A
:104750004C69627261726965735C53544D333246C1
:104760003130785F5374645065726970685F447269
:10477000697665725C7372635C73746D3332663133
:1047800030785F74696D2E630000000070B50446D8
:104790000D461D48844217D0B4F1804F14D01B48F9
:1047A000844211D01A4884420ED01A4884420BD059
:1047B0001948844208D01948844205D018488442D8
:1047C00002D01848844200D104E040F64A1116A0F5
:1047D00001F042FB2DB1042D03D0082D01D00C2D8A
:1047E00000D104E040F64B110FA001F035FB208B07
:1047F0004FF2FF3108402083208B4FF6FF7101EA12
:1048000005210843208370BD002C014000040040B6
:1048100000080040000C004000340140004C014002
:1048200000180040004001404C6962726172696585
:10483000735C53544D3332463130785F5374645057
:1048400065726970685F4472697665725C737263E1
:104850005C73746D3332663130785F74696D2E63CA
:104860000000000070B504460D46174884420ED083
:10487000B4F1804F0BD01548844208D014488442CC
:1048800005D01448844202D01348844200D104E089
:104890004FF4166111A001F0DFFA2DB1042D03D001
:1048A000082D01D00C2D00D104E040F661110BA0C1
:1048B00001F0D2FAA08B4FF6F3710840A083A08BD1
:1048C0002843A08370BD0000002C0140000400407C
:1048D00000080040000C0040003401404C69627246
:1048E00061726965735C53544D3332463130785F81
:1048F0005374645065726970685F4472697665725A
:104900005C7372635C73746D3332663130785F74DC
:10491000696D2E630000000070B504460D4619480D
:1049200084420ED0B4F1804F0BD01748844208D097
:104930001648844205D01648844202D01548844265
:1049400000D104E040F6761113A001F085FA2DB1F4
:10495000042D03D0082D01D00C2D00D104E040F629
:1049600077110DA001F078FAA08B4FF2FF310840CB
:10497000A083A08B4FF6FF7101EA05210843A083B5
:1049800070BD0000002C0140000400400008004001
:10499000000C0040003401404C696272617269652C
:1049A000735C53544D3332463130785F53746450E6
:1049B00065726970685F4472697665725C73726370
:1049C0005C73746D3332663130785F74696D2E6359
:1049D0000000000070B504460D4600264A48844297
:1049E0002FD0B4F1804F2CD04848844229D0484879
:1049F000844226D04748844223D04748844220D06E
:104A0000464884421DD0464884421AD045488442D4
:104A100017D04548844214D04448844211D04448B9
:104A200084420ED0434884420BD04348844208D08D
:104A30004248844205D04248844202D041488442E0
:104A400000D103E0E72140A001F006FA688858B1E0
:104A50006888102808D06888202805D068884028F1
:104A600002D06888602800D103E0E82136A001F078
:104A7000F3F9E88838B1E888B0F5807F03D0E8889A
:104A8000B0F5007F00D103E0E9212FA001F0E4F9A7
:104A900026881D4884420ED0214884420BD0B4F1B0
:104AA000804F08D01948844205D01948844202D06A
:104AB0001848844204D14FF68F7006406888064338
:104AC0001548844207D01548844204D04FF6FF4071
:104AD0000640E88806432680A888A0852888208587
:104AE000094884420BD00E48844208D013488442BF
:104AF00005D01348844202D01248844201D1287A5A
:104B000020860120A08270BD002C014000040040DE
:104B100000080040000C004000100040001400405D
:104B200000340140004C014000500140005401405D
:104B300000180040001C00400020004000400140E0
:104B400000440140004801404C696272617269652D
:104B5000735C53544D3332463130785F5374645034
:104B600065726970685F4472697665725C737263BE
:104B70005C73746D3332663130785F74696D2E63A7
:104B8000000000004FF6FF71818000210180C1808C
:104B9000418001727047000010B50F48007818B1CD
:104BA00000200E4908600DE001200C4908600C4807
:104BB0000068401E0A4908600846006810B90520D0
:104BC000FEF76CFD0448007808B9012000E00020E1
:104BD0000149087010BD00001C0000208C81224299
:104BE000200000200F480078401CC0B20D4908701A
:104BF0000A2190FBF1F201FB12000A4908700846F5
:104C00000078002801DD012000E00020064908604E
:104C1000064800680649A1F8A40006480068C1F8E3
:104C2000A00070479E01002080812142081C0140A5
:104C3000C80300200C14014010B513480078002868
:104C400010DD11480078401E0F49087008460078B2
:104C500040B90E480078002804DD01F00DF900206D
:104C60000A4908700A48007800280CDD08480078D6
:104C7000401E074908700846007820B90020054901
:104C80000870FEF753FB10BD000000200900002053
:104C9000010000200A0000202DE9F05FDFF8C49039
:104CA000D9F84400C11700EB11714FEA211A4846A8
:104CB000D0F8A8B02C490988A1EB0A0101EB410109
:104CC000490001EB8101092291FBF2F000EBD07168
:104CD0004C10FDF7B1FA05460E46FDF7E3FA07461C
:104CE0002A46334602F0E0F9204A03C22048006811
:104CF00000280BDD1E480068401C1D490860002488
:104D000008460068322801DD0020086000224FF0CC
:104D10004043164903C902F04BF812D2FDF7C2FA1C
:104D200005460022134B02F043F80AD2FDF784FA3D
:104D300005460022104B02F075F902D201200C4901
:104D40000860094800880D490860142C02DA002C1C
:104D500000DD1424204602F000F80546FEF7A4FB0F
:104D6000BDE8F09FC803002038000020700000203C
:104D70007800002000005940000049407C000020DD
:104D800010B5414CA4F1E800D0F8B4003F49884286
:104D900003DD0020FEF7D4FA10BDE168216172B690
:104DA000206801683848E838D0F8B400081A4FF491
:104DB0008D7190FBF1F0401DE06062B6D4E9031004
:104DC000081A6061D4E9021088423BDAE06800EB1F
:104DD0008000C000322190FBF1F020626169E06840
:104DE000484300281BDBE06800EB8000C000322154
:104DF00090FBF1F0A1690844A0612821A06990FB13
:104E0000F1F0C82802DD4FF4FA50A0612821A06912
:104E100090FBF1F010F1C80F01DA1D48A0612821C4
:104E2000A06990FBF1F0216A08442062616901EBFE
:104E30008101C800C11700EB9171226A02EBA10148
:104E4000216201E0FF2020626068B0F900004FF4A9
:104E50007A71484390FBF1F06169884201DD0020DE
:104E60002062206A002801DA00202062206AFF28E0
:104E700001DDFF20206294F82000FEF761FA206A2D
:104E8000E06100BF88E70000B0040020C0A233004A
:104E9000C0E0FFFF0C49888C0C49D1F8D820C1F83C
:104EA000D4200B4909880B4A126801EB02420749DA
:104EB000C1F8D820D1F8D820D1F8D410511A064A18
:104EC000116000BF7047000000080040C8030020C8
:104ED000240800402C0000203000002070B513484A
:104EE00005681348807B00B970BD12480078B8B9D6
:104EF0000E480068012813D10D4890F81A0178B9BE
:104F00000B4890F8190140B1094890F81901001DAB
:104F1000C4B22046FDF7A8FD02E00120FDF7A4FD84
:104F2000024800680349087000BFDDE700812342A2
:104F3000C8030020280000202DE9FF41624890F8B6
:104F400020010E287ED2DFE800F007091A1C1E207F
:104F5000222C3343556D818C00BFA9E05A4890F84C
:104F6000214190F83401A04207D0574880F83441DD
:104F7000014691F83401FEF7C3F900BF98E000BF85
:104F800096E000BF94E000BF92E000BF90E00120F7
:104F90004D4981F837014FF47A710D20FBF73CFE43
:104FA00086E0494991F82101FDF7A0FC00BF7FE0B0
:104FB00000BF454890F82101002805DD424991F8DD
:104FC0002101FDF751FD01E0FEF73EFB00BF6FE060
:104FD0000F203D4981F835010846807B18B191F8D2
:104FE0002101FDF741FD4FF47A710920FBF714FE12
:104FF00000BF5DE0FEF7F8FA0120FDF777FC09201D
:10500000FEF74CFB0A20FEF749FBFEF7D5FA01201C
:10501000FDF76CFC2D48FEF727FB00202A4981F89C
:10502000350145E000BF284890F8210158B12648D5
:1050300090F8231190F8220101EB00252846FEF795
:1050400021FA02E029E0FEF7B7FA31E000BF1E497D
:1050500091F8210101F112023C31FBF79FFE00BFE4
:1050600026E01B48011D0EC900698DE80E00039063
:10507000102269461748FBF7E9F868B1DDE90273C9
:105080003A46DDE900512846FBF708FE00F0D2FE63
:1050900010489DE82E002EC00AE000BF0A4890F894
:1050A000200100F0800008B100BF00E000BF00BF99
:1050B00000BF054890F8200140F08000024981F8C7
:1050C0002001BDE8FF810000C80300205800002037
:1050D000E8040020D00D002010B52C48007810B94D
:1050E00001F038F851E02A480078002814DD002447
:1050F00010E004EB8400274901EB8000406824495C
:105100000978401A04EB8401224A02EB81014860CD
:10511000601CC4B20D2CECD300201C4908701C4943
:10512000087000242FE004EB84001A4911F82000D5
:1051300000B926E004EB8400164901EB80004068CA
:10514000401E04EB8401134A02EB810148600028F1
:1051500016DC04EB8400114601EB8000406804EB90
:10516000840102EB81018968084404EB840102EBAD
:105170008101486004EB840102EB810108698047EA
:1051800000BF601CC4B20D2CCDD310BD9C0100200B
:105190009D0100209800002010B500BF304890F815
:1051A0003701062855D2DFE800F054032036445575
:1051B0000120FDF79BFB2A4A123202F12A0100204E
:1051C000FBF7ECFD4FF4FA710120FBF74FFD0020D7
:1051D000FDF77AFB0020FDF7B7FD0020FBF7FCFD93
:1051E00002201F4981F8370138E01D4890F8DC00A3
:1051F00001280FD11A4890F8DD0058B91848807B73
:1052000020B90520164981F8370103E0032014492D
:1052100081F8370122E0124890F8DC00012807D11C
:105220000F49487CFDF720FC04200D4981F8370127
:1052300014E00B4890F919010949497C884207D1CB
:10524000074890F81A0118B90520054981F8370177
:1052500004E000BF0D20FEF721FA00BF00BF10BD23
:10526000C803002010B5424890F8DE0010B9FDF7E1
:1052700049FD68B13E4890F8DE00012802D1FDF7F3
:1052800051FD28B1FDF73EFD20B9FDF74BFD08B9F2
:10529000FEF7AAF9FCF7A0FF354890F8DE000128D8
:1052A00016D13348D0F8E000401E3149C1F8E00083
:1052B0000846D0F8E00010F1C80F21DC012081F889
:1052C000DC00FEF791F964210A20FBF7CFFC17E020
:1052D0002748D0F8E000401C2549C1F8E000084606
:1052E000D0F8E010D0F8E400814209DB0420204926
:1052F00081F8DC00FEF778F964210120FBF7B6FCA9
:105300001B48D0F8E010D0F8E40081422ED11848B4
:1053100000884FF47A7148430A2190FBF1F0322162
:1053200090FBF1F11248D0F8E400814207D102204D
:105330000F4981F8DC0000BFFEF756F916E00C4873
:1053400040884FF47A7148430A2190FBF1F03221F2
:1053500090FBF1F10648D0F8E400814206D1032029
:10536000034981F8DC0000BFFEF73EF910BD0000E4
:10537000C803002010B51E480068401E1C49086084
:105380001C4890F81801012818D01A4890F8190103
:10539000A0B119480078012810D11848006868B9F0
:1053A000144890F919011349097C90FBF1F201FBB3
:1053B0001200401C41B20F4880F8191110480068D3
:1053C00018B901210B4880F819110C4800680A49E6
:1053D0000870084890F91901064991F81811884297
:1053E00003D003480068002801DCFEF72DF910BD4A
:1053F00010000020C80300200C0000201081234270
:10540000148123422DE9F84FFCF702FF344908606C
:1054100034480068401E33490860FCF7FDFA002854
:105420004AD0314890F818B1007C00900024ABF1CC
:1054300001002E4931F8100029490968A1EB000A42
:105440002B48006801F089FC05460E46504601F0E5
:1054500084FC21F0004107462A46334601F0A8FCAF
:1054600006D24FFA8BF1204880F81911FEF7DCF8CC
:1054700000241DE01D4830F8140019490968A1EB0B
:1054800000091B48006801F068FC05460E464846C6
:1054900001F063FC21F0004107462A46334601F043
:1054A00087FC04D2601C41B20F4880F81911641CBB
:1054B00000988442DEDB00BF0A48006800280CDA4E
:1054C0000021094880F819114FF47A710120FBF787
:1054D000CDFBFCF7A7FAFEF7A7F8BDE8F88F0000B0
:1054E0001400002010000020C80300209C050020AC
:1054F000180000202DE9F0419548066C476CD0F863
:10550000A8500446D4F83801401CC4F83801D4F837
:105510003C01401CC4F83C01204690F8350110289D
:105520007DD2DFE800F0080C456A98C1E27CEA7C95
:105530007C7C345980F50920FEF7B0F804E10020A6
:10554000C4F83801C4F83C010220FDF7CFF98148C6
:10555000FEF78AF80020FDF795FF0A210846FBF7C1
:105560005BFB0120FDF7B0F90120FDF7EDFB00200A
:10557000C4F838010C2084F83501FDF755FEFDF71D
:10558000DFF84FF4FA710120FBF770FBDCE07048A4
:1055900090F8DC00022804D06D4890F8DC00042864
:1055A00005D10020C4F83801022084F83501CBE091
:1055B000E0884FF47A71484390FBF1F0D4F8381149
:1055C000884208D20320FDF791F90D2084F83501B7
:1055D0000020C4F83801B7E05D4890F8DC000328EB
:1055E00004D05B4890F8DC00042805D10020C4F802
:1055F0003801032084F83501A6E020894FF47A7140
:10560000484390FBF1F0D4F8381188420AD20020C8
:10561000C4F838010E2084F83501042000E092E03F
:10562000FDF764F990E04A4890F8DC00042803D0C4
:10563000D4F838011E280DD9D4F838011E2803D912
:1056400064210A20FBF712FB042084F835010020B6
:10565000C4F8380178E03E498989D4F83C01884291
:1056600005D33C48FEF700F80020FCF7E1F994F878
:105670003501042817D1B54203DD3648FDF7F4FFA4
:1056800011E0BD420FDA334890F90000401C50B9D8
:105690006089642200FB02F100232F4A0120FDF7FC
:1056A00051FF2C4908704FE00A20FDF7F7FFFDF786
:1056B00083FF274890F8DC00012803D0D4F8380194
:1056C000462811D94FF4FA710220FBF7CFFA20488F
:1056D000807B30B1E07B84F83601082084F8350106
:1056E00002E0002084F835012EE0194890F81A01F4
:1056F00010B9002084F8350126E094F83611481ED0
:1057000084F8360111B9062084F835011CE0FFE762
:105710000120FDF7D9F80120FDF716FB0C48807B2E
:1057200010B9012084F83501094890F8181190F952
:105730001901814206D1064890F81A0110B90120DA
:1057400084F8350100E000BF00BFBDE8F081000033
:10575000C803002058000020311A000870B5174C0B
:10576000002527E0207800B921E0A068401EA06055
:1057700000281BDC607820B101280DD0022811D14F
:1057800002E00020207010E0D4E901100844A0607D
:10579000D4E90310884708E0D4E9031088470020C3
:1057A000207002E00020207000BF00BF00BF681C16
:1057B000C5B21434052DD5DB70BD0000DC1F002000
:1057C00010B540F22551244800F0ACF870B1032028
:1057D000224908702048001D0088C1B22048027884
:1057E0000078401C1E4B18701E48815440F22771EF
:1057F000194800F097F8F0B11B4800781B49097868
:1058000088420CDA1A4818490978405C1249091D87
:10581000088015480078401C134908700BE00022EE
:1058200040F227710C4800F023F9012240F2266172
:10583000094800F01DF940F22661074800F072F8AF
:1058400040B1002240F22661034800F011F9012026
:105850000849086010BD0000003801400000002029
:1058600009000020B40200200A00002008000020E7
:10587000B4010020B001214270B504460D46154820
:1058800084420BD01448844208D01448844205D086
:105890001348844202D01348844200D104E04FF4FC
:1058A000B17111A000F0D8FA0DB1012D00D104E0C2
:1058B00040F263110CA000F0CFFA25B1A08940F4AA
:1058C0000050A08104E0A0894DF6FF710840A0813E
:1058D00070BD000000380140004400400048004016
:1058E000004C0040005000404C6962726172696572
:1058F000735C53544D3332463130785F5374645087
:1059000065726970685F4472697665725C73726310
:105910005C73746D3332663130785F7573617274A5
:105920002E6300002DE9F04705460C4600270026AF
:10593000B046B1463A4885420BD03A48854208D035
:105940003948854205D03948854202D038488542D9
:1059500000D104E040F2C13136A000F07DFA282CDD
:1059600020D040F2277084421CD040F2266084424E
:1059700018D040F22550844214D040F22440844292
:1059800010D040F6460084420CD040F66A108442A3
:1059900008D0B4F5587F05D0B4F5187F02D0B4F51F
:1059A000B07F00D104E040F2C23122A000F054FAEE
:1059B00040F66A1084420ED11948854205D0194834
:1059C000854202D01848854200D104E040F2C63139
:1059D00018A000F041FAC4F3421804F01F06012099
:1059E00000FA06F6B8F1010F02D1A889064007E0D7
:1059F000B8F1020F02D1288A064001E0A88A0640C9
:105A00002712012000FA07F7288807401EB117B1B6
:105A10004FF0010901E04FF000094846BDE8F0876A
:105A2000003801400044004000480040004C004065
:105A3000005000404C69627261726965735C535436
:105A40004D3332463130785F5374645065726970FB
:105A5000685F4472697665725C7372635C73746DBF
:105A60003332663130785F75736172742E63000073
:105A70002DE9F04705460C4617464FF00008C24690
:105A8000C1460026384885420BD03848854208D0A8
:105A90003748854205D03748854202D0364885428E
:105AA00000D104E040F2891134A000F0D5F9282C8F
:105AB00019D040F22770844215D040F2266084420B
:105AC00011D040F2255084420DD040F2244084424F
:105AD00009D040F64600844205D040F66A10844260
:105AE00001D0602C00D104E04FF4C57123A000F078
:105AF000B3F90FB1012F00D104E040F28B111FA0C8
:105B000000F0AAF940F66A1084420ED11648854288
:105B100005D01648854202D01548854200D104E0E0
:105B200040F28F1115A000F097F92E46C4F34218E9
:105B300004F01F0A012000FA0AF9B8F1010F01D19F
:105B40000C3605E0B8F1020F01D1103600E0143632
:105B500027B1306840EA0900306003E0306820EA8D
:105B600009003060BDE8F087003801400044004083
:105B700000480040004C0040005000404C696272F8
:105B800061726965735C53544D3332463130785FCE
:105B90005374645065726970685F447269766572A7
:105BA0005C7372635C73746D3332663130785F7529
:105BB000736172742E6300002DE9F04786B00546CC
:105BC0000C460026B24600BFB14600276B4885420E
:105BD0000BD06B48854208D06A48854205D06A4898
:105BE000854202D06948854200D103E0B82168A00F
:105BF00000F032F9206820B174492068884200D250
:105C000003E0B92162A000F027F9A08818B1A088AC
:105C1000B0F5805F00D103E0BA215DA000F01CF96F
:105C2000E08858B1E088B0F5805F07D0E088B0F533
:105C3000005F03D0E088B0F5405F00D103E0BB21F6
:105C400053A000F009F9208938B12089B0F5806FA0
:105C500003D02089B0F5C06F00D103E0BC214CA077
:105C600000F0FAF860894FF6F371084010B96089C6
:105C700000B103E0BD2146A000F0EEF8A08958B1C4
:105C8000A089B0F5807F07D0A089B0F5007F03D050
:105C9000A089B0F5407F00D103E0BE213CA000F018
:105CA000DBF8A08968B13548854205D03448854283
:105CB00002D03448854200D103E0C22134A000F074
:105CC000CBF82F462E8A4CF6FF700640E08806433C
:105CD0002E82AE894EF6F3100640A0882189084333
:105CE000618908430643AE81AE8A4FF6FF40064005
:105CF000A0890643AE8201A8FDF788F91F488742B4
:105D000002D1DDF810A001E0DDF80CA0A88900F4B4
:105D1000004040B10AEBCA0000EB0A1021684900BC
:105D2000B0FBF1F807E00AEBCA0000EB0A102168AB
:105D30008900B0FBF1F86420B8FBF0F006013009EF
:105D4000642101FB1089A88900F4004040B1322091
:105D500000EBC900B0FBF1F000F00700064308E0DB
:105D6000322000EB09106421B0FBF1F000F00F00CD
:105D700006432E8106B0BDE8F087000000380140E0
:105D80000044004000480040004C004000500040EB
:105D90004C69627261726965735C53544D3332466B
:105DA0003130785F5374645065726970685F447213
:105DB000697665725C7372635C73746D33326631DD
:105DC00030785F75736172742E63000021AA4400FD
:105DD00000BFFEE710B500BF1548FDF717F900F04A
:105DE00033FCFCF7ADFBFCF703FD4FF47A70FBF7D7
:105DF000D8FBFCF731FCFCF7F9FA4FF47A7101207B
:105E0000FAF734FFFCF796FBFCF79AFCFDF7D4FB9E
:105E1000FCF716FCFCF7E0FCFDF7BEFB642101205B
:105E2000FAF724FFFCF74EFD0148FDF7EFF810BD2F
:105E3000A001002010B54E21064800F0CFF804461E
:105E400004485038A0F89E40102250215030FBF7F3
:105E5000E9FB10BD1804002000BF00BFFEE70000F2
:105E600000200349086006200249087070470000BE
:105E7000B00121420100002070B555480078554915
:105E800091F83411884204D051480078FF2800D09E
:105E900070BD5148007804287EDD4D4840780528C3
:105EA00014D008DC01280DD002280CD003280BD018
:105EB000042872D109E0062809D00F2845D01028FF
:105EC000F7D153E000BF00BF00BF00BF00BF424892
:105ED0000078082838DB06213D4800F07FF80546A9
:105EE0003B48C0793A49897900EB0120A84228D182
:105EF00037484078012802D100F0D2F921E0344837
:105F00004078022802D1FDF71FF91AE030484078A6
:105F1000032802D100F086FA13E02D4840780428C7
:105F200002D100F02DFA0CE029484078052802D172
:105F300000F070F805E026484078062801D100F00E
:105F400075F90020244908703EE02148847909341D
:105F500021480078A04208DBA01E81B21C4800F056
:105F60003DF8054600201C4908702DE0184840798E
:105F70001749097900EB012084B24FF6FF7000EA5F
:105F8000440404F1090084B213480078A04219DBEC
:105F9000A01E81B20E4801E017E014E000F01EF8E8
:105FA0000546601E0A49095CA01E094A105C01EB07
:105FB0000020A84203D100F0EBF8FEF7BDFF00205F
:105FC0000549087000E000BF00BF00BF60E70000A7
:105FD000B4020020C80300200900002070B502466A
:105FE0000C46FF25FF2309E012F8010B80EA0501AA
:105FF0000648405C80EA03050548435C201EA4F186
:106000000106B4B2F0D143EA052070BD7C720008ED
:106010007C7300082DE9F0411048C778B84606792E
:10602000FF2E01D1012501E006B90025E9B2404665
:1060300000F04AFA002405E00848005D08490855C8
:10604000601CC4B2074800788442F5DB054800783C
:1060500005490870FFF704FFBDE8F081B402002095
:10606000B40100200900002008000020F0B503461C
:106070000A46002400250026D9B20846CF1701EBB6
:1060800017773F11A1EB0717B9B20846CF1701EBFD
:106090005777FD10CF1701EB5777FF10A1EBC7061D
:1060A00009480068094FC7F8A00007F1A0042C4474
:1060B00020780127B740384010B10120107001E06E
:1060C000002010700120F0BD0C140140C803002016
:1060D00030B502460020054B054D2D681D80C2F3EA
:1060E0000B0433F814500D8030BD00006C04002008
:1060F000081C0140F0B503460A460024002500268E
:10610000D9B20846CF1701EB5777FD10CF1701EB37
:106110005777FF10A1EBC706064C2C4420780127C7
:10612000B740384010B10120107001E0002010701D
:106130000120F0BD6C04002010B502460020C2F31F
:106140000B03034C246834F813400C8010BD00008E
:1061500004000020704700002DE9F04104460D4680
:1061600000BF0022054B2046294600F05DFE064692
:106170000022034B00F000FCBDE8F08100FEAF40C0
:1061800000407F40FFF726FE01E0FEF7A5FFFCE799
:106190002DE9F0432148C0782049897800EB01209F
:1061A00085B2C5F30B081D484679002417E0082086
:1061B00000EB44001949085C072101EB4401174A30
:1061C000515C00EB01201FFA80F94946404600F07F
:1061D000CBF9601C84B208F101001FFA80F8B442C8
:1061E000E5DB0F4890F834010E4908701020487024
:1061F00028128870CD70301208714E71062109483E
:10620000FFF7ECFE0746381206498871CF71082067
:1062100005490870FFF724FEBDE8F083B4020020B2
:10622000C8030020B40100200800002070B5184801
:10623000C0781749897800EB0120C4B2144840792E
:106240001349097900EB012085B272B62946204630
:1062500000F08AF962B60F4890F834010E490870D0
:1062600006204870201288700846C47028120871F1
:106270004D7106210848FFF7B1FE06463012064967
:106280008871CE71082005490870FFF7E9FD70BDDF
:10629000B4020020C8030020B40100200800002040
:1062A0002DE9FC4F00200090314890F803B0D8460B
:1062B00045792846E91705EB5171CC10E91705EB34
:1062C0005171C910A5EBC10109B1601CC4B200270E
:1062D0002CE0F81CC6B200202649885582461BE0F7
:1062E00001A94046FFF7C2FE2248805D9DF80410D8
:1062F00001FA0AF108431F49885508F1010000F02E
:10630000FF080BEB0500404502DC0120009006E091
:106310000AF1010000F0FF0ABAF1080FE0DB00BF4C
:106320000098012800D103E0781CC7B2A742D0DB57
:1063300000BF114890F834010E49087001204870E0
:1063400008468470E01CC4B221460A48FFF746FEA6
:1063500081464FEA292007490855601CC4B201F85C
:106360000490601C05490870FFF77AFDBDE8FC8FBA
:10637000B4020020B4010020C8030020080000205F
:106380002DE9F843002000902248C07821498978FF
:1063900000EB012000F0FF0847461E4890F80590EA
:1063A0004FEA4960040E72B6002512E0694638468D
:1063B000FFF78EFEBDF800000112174AE81C1154C9
:1063C000BDF80000C1B2281D1154A81C85B2781C6C
:1063D000C7B2A542EADB62B6104890F834010E4914
:1063E00008700420487008468470E01CC4B221463E
:1063F0000948FFF7F3FD0646301207490855601CAF
:10640000C4B20E55601C06490870FFF729FDBDE8AF
:10641000F8830000B4020020B4010020C80300206B
:10642000080000202DE9F843002000902248C078A1
:106430002149897800EB012000F0FF0847461E48FB
:1064400090F8059002244FEA4960040E72B60025C8
:1064500012E069463846FFF76FFEBDF800000112F2
:10646000164AE81C1154BDF80000C1B2281D115491
:10647000A81C85B2781CC7B2A542EADB62B61048F8
:1064800090F834010D490870032048700846847064
:10649000E01CC4B221460948FFF7A0FD06463012B1
:1064A00006490855601CC4B20E55601C05490870A9
:1064B000FFF7D6FCBDE8F883B4020020B401002049
:1064C000C8030020080000202DE9F04103460C46D7
:1064D0004FF0000C002200270025D9B208464FEAF1
:1064E000E17801EB18784FEA2818A1EB08181FFA99
:1064F00088F108464FEAE17801EB58784FEAE8075F
:106500004FEAE17801EB58784FEAE808A1EBC805BB
:1065100013480068DFF84C80C8F8A00008F1A0021A
:106520003A444CB110784FF0010808FA05F840EAF7
:106530000800107000BF08E010784FF0010808FA5A
:1065400005F820EA0800107000BF16780548D0F85A
:10655000A000DFF80C80C8F800006046BDE8F081BC
:106560000C140140C803002010B50246002072B68A
:10657000C2F30B03024C246824F8131062B610BD5A
:10658000040000202548806940F004002349886108
:106590002348244908602448091D08601F48806971
:1065A00040F008001D4988612048214908602148C1
:1065B000091D08601948806940F01000174988617A
:1065C0004FF4C6001C4908604FF48000486013482F
:1065D000806940F02000114988614FF0113017495F
:1065E00008600020091D08600C48806940F04000E8
:1065F0000A4988614FF0443011490860091D08605C
:106600000648806940F08000044988614FF0883076
:106610000C490860091D0860704700000010024026
:106620004444131400080140B44F434422444444FA
:10663000000C014044BBB44B001001400014014069
:1066400000180140001C014010B500BF1F48204940
:1066500048602048086000BF00BF1D48006800F087
:1066600002000028F9D000BF1948006800F400308B
:106670000028F9D000BF1648006800F0007000281C
:10668000F9D000BF1248406800F00C000828F9D18A
:1066900000BF00BF00201049086000BF00BF41F6E6
:1066A00057304FF0E02148610220086100208861E6
:1066B0000846006940F00100086100BF00BF00BF4C
:1066C000FFF760FF00F00AF810BD00000228150077
:1066D000001002408300090108ED00E0464880698F
:1066E00040F00100444988614448406820F00400BB
:1066F000424948604048806940F004003E49886152
:106700003F48006820F47F603D4908600846006803
:1067100040F0B00008600846006840F480600860FF
:106720003548806940F480403349886140F2B25076
:10673000344908800020091D0880091D0880081FB1
:106740000088091F088000202E490C3108802D4840
:10675000001D008840F00C002A49091D08800846E9
:10676000008840F4005008802348806940F0010010
:10677000214988612148406820F030001F49486065
:106780001D48806940F008001B4988611E48006868
:1067900020F47F401C4908600846006840F43060DF
:1067A00008600846006840F4804008601248C069EC
:1067B00040F480201049C86141F2C9601349088043
:1067C0000020091D0880091D0880081F0088091F76
:1067D000088000200D490C3108800C48001D0088FD
:1067E00040F00C000949091D08800846008840F463
:1067F0000050088070470000001002400000014077
:106800000408014008380140040C014008480040D9
:1068100010B591EA030F48BF83F0004300F14C84A8
:10682000841A71EB030C05D2121943EB0C03001B05
:1068300061EB0C01DFF824E14FEA1154A4EB135C87
:106840001EEA430F18BF9EEA445F73D023EA0E038B
:10685000DCF1200E21EA045143F4801332D322FAF2
:106860000CFE10EB0E0023FA0CFE41EB0E01CCF1F6
:10687000200E03FA0EFE10EB0E0051F10001B1F5EF
:10688000801FCCF1200E32D201EB045112FA0EF22D
:10689000BDE8104058BF7047401C38BF5FEA420255
:1068A00018BF7047002814BF20F0010041F100011B
:1068B0004FEA410313F5001F38BF7047A1F1C041F3
:1068C00000F0AABB012A43EB0302ACF1200CDCF17F
:1068D0001F0E32BF4FF0000E23FA0CF310EB030033
:1068E00041EB0451B4EB115FD0D0A1EB045101F5A1
:1068F000801149085FEA300001EB04510ED350F1DA
:10690000000038BF12FA0EFE08D1BDE81040C9E7FA
:10691000401C38BF5FEA4202CAD1C3E7BDE810405D
:106920004FEA410313F5001F38BF7047A1F1C04182
:1069300000F072BB9EEA445F08D011EA5E0FBDE82A
:10694000104004BF01F0004100207047BDE8104036
:1069500070B500F013FB00BF64FBBE3E0000E0FF1B
:10696000491058BFC1F140415B1058BFC3F14043CB
:106970008B42EFF3008070472DE9C04130B4DFF85F
:10698000A0C23CEA111418BF3CEA131400F0EC80DA
:1069900081EA03051CEA111444EAD57418BF1CEA05
:1069A000131500F0C780A4EB05044FF0004545EA3D
:1069B000C12145EAC32341EA505143EA525304F14D
:1069C0007F74994204F500344FEAC0204FEAC22296
:1069D00008BF904200F09C804FEA13650FF240160A
:1069E000765D4FEA134506FB05F7C7F1807706FB96
:1069F00007F74FEAD737A7FB03687642C8F5803818
:106A0000A7FB06CE38BFA8F1010807FB08E64FF048
:106A1000000EA6FB028CE6FB03CEDCF1000CCEF1EF
:106A2000004E38BFAEF1010EA6FB0C584FF0000728
:106A30004FF00005E6FB0E87A1FB08C6A0FB07CEC2
:106A400016EB0E0645F10005E1FB076515F1E04E7A
:106A50007EBFA4F580345FEA46066D4116F18007DB
:106A600045F100054FEA17274FEA066647EA056732
:106A7000A6F1DE46B6F1805F4FEA15251FD93846EC
:106A800024F0010C05EBC471BCF1FE6F01EB0C119D
:106A900002D8F0BCBDE8008124425CBF01F5801E35
:106AA0009EEAC47F02D4F0BCBDE80081244238D401
:106AB000F0BCA1F1C041BDE8004100F0ADBA4FEA21
:106AC000D22242EA43524FEAD323A7FB02864FEA7F
:106AD000D02040EA415007FB03661EEA0E0F4FEA42
:106AE000D12105FB026658BFA6EB0056B6EB005657
:106AF0004FEA520E4EEAC37E18EB0E0E56EB530EC3
:106B0000BDD518EB02085E417F1C55F10005B6E7C4
:106B10004FF480154FF000074FF000064FF00008CB
:106B2000ADE7F0BC4FF0000001F1C04101F00041C1
:106B3000BDE8008111EA0C1F0CEA131500D00CE02F
:106B400013EA0C1F00F025804FF00000F0BC81EA32
:106B5000030101F00041BDE80081F0BCBDE8004147
:106B600081EA030100F058BAF0BCBDE8004170B5FD
:106B700000F004FA097EFC3E00F007B881EA030148
:106B80004FF0000001F00041704781EA030100F07E
:106B900043BAF0BCBDE800414FF000002149704706
:106BA000FFFDFBF9F7F5F4F2F0EEEDEBE9E8E6E4D2
:106BB000E3E1E0DEDDDBDAD8D7D5D4D3D1D0CFCD59
:106BC000CCCBCAC8C7C6C5C4C2C1C0BFBEBDBCBB92
:106BD000BAB9B8B7B6B5B4B3B2B1B0AFAEADACAB8D
:106BE000AAA9A8A8A7A6A5A4A3A3A2A1A09F9F9E67
:106BF0009D9C9C9B9A999998979796959594939319
:106C0000929191908F8F8E8E8D8C8C8B8B8A8989AF
:106C10008888878786858584848383828281818032
:106C20000000FF070000F87F51EA030C17D41CF5A1
:106C3000801F58BFBCF5801F00F10680994218BF25
:106C4000704708BF9042704707D711F5801F58BFA3
:106C500013F5801F19D499427047894270471CF57B
:106C6000801F08D5BCF5801FF7D58B4218BF704731
:106C700008BF824270474FF4001C1CEB410F38BF25
:106C80001CEB430F01D28B42704770B500F076F9D0
:106C9000922449004FF000514FF08053FFF760BE3F
:106CA0004FEA41034FEA5353A3F58063D3F11E0328
:106CB000C8BFD3F1210C0CDD4FF0004242EAC122E3
:106CC00042EA505232FA03FC8CEAE17CACEBE17010
:106CD0007047102BC4BF0020704703F5787CBCF1CF
:106CE000FF3F04D06FF0004282EA2100704770B588
:106CF00000F044F94992248000207047F2E7000038
:106D00004FEA1153A3F58063D3F11E03A8BFD3F15B
:106D1000200C08DB4FF0004242EAC12252EA5052F6
:106D200032FA03F0704709420BD4102BC4BF002085
:106D3000704703F5787CBCF1FF3F05D04FF0FF3082
:106D400070474FF00000704770B500F017F900BFB2
:106D50004992248000207047F0E710F0004248BFBD
:106D60004042B0FA80F310FA03F10AD0C3F11D03D8
:106D700003F580634FEA415002EB035202EBD1214D
:106D800070474FF000007047B0FA80F310FA03F13B
:106D90000AD0C3F11D0303F580634FEA41504FEA67
:106DA000035202EBD12170474FF000007047000002
:106DB00051EA030C17D41CF5801F58BFBCF5801F87
:106DC00000F10680994218BF704708BF9042704793
:106DD00007D711F5801F58BF13F5801F19D49942AA
:106DE0007047894270471CF5801F08D5BCF5801F8D
:106DF000F7D58B4218BF704708BF824270474FF4E7
:106E0000001C1CEB410F38BF1CEB430F01D28B421F
:106E1000704770B500F0B2F8922449004FF000516D
:106E20004FF08053FFF79CBDDFF848C170B51CEAF6
:106E3000111E1EBF1CEA13159EEA0C0F95EA0C0FDB
:106E400000F06F8081EA030423EA4C134EEAD47EFB
:106E500021EA4C1141F4801143F48013AE44A1FBAC
:106E6000024CA0FB0365AEF17F7E361955EB0C0595
:106E7000A1FB034C4CF10003A0FB021C16EB0C061B
:106E8000654153F10003094218BF46F0010613F4AF
:106E9000007F0BD14FEA03314FEA0530340341EA5A
:106EA000155140EA16506FF003020AE04FEAC32181
:106EB0004FEAC520F40241EA555140EA56506FF0BE
:106EC000020202EB2E4201EB025585EACE710AD096
:106ED0005FEA440C18BF24F0004450F1000041F177
:106EE000000120EAD47040F2FE7C624500D270BD01
:106EF000A84214BF4FF080444FF04044002E08BF1A
:106F00000024BEF1806FA8BFA1F1C041BDE8704070
:106F100080F282804FF0000001F1C04101F0004199
:106F200070479EEA0C0F0CEA131518BF95EA0C0F78
:106F300006D04FF0000081EA030E0EF0004170BD54
:106F400000F01CF88900013E00F007B800F009B815
:106F50004FEA430C5FEA5C5C08D081EA030100F071
:106F60005BB84FEA410C5FEA5C5CF6D14FF0000081
:106F7000014970470000FF070000F87F0EF1020E84
:106F80002EF0030E5EF8046B364205D4012A43EB63
:106F9000030515F5001F12D8012841EB010C1CF563
:106FA000001F0CD80ED14FEAD17C15F5001F0CEB59
:106FB0004C0C0CF1020C08BF4CEBD37C04E04FF0FE
:106FC000080C01E04FEAD37C0CEB4C0526FA05F6E1
:106FD00006F00706B6F1040C06D20EEB860CBDE8EF
:106FE00070404CF0010C6047DFE80CF0090B020226
:106FF0004FF000414FF00000A1F5002170BD19468F
:107000001046012851EB010418BFD4F5001484BFC9
:10701000002001F0004170BD0808A0F500114FEA02
:107020003101704753EA010C17D41CF5801F58BF7B
:10703000BCF5801F00F106808B4218BF704708BF67
:107040008242704707D713F5801F58BF11F5801F84
:1070500019D48B4270479B4270471CF5801F08D59E
:10706000BCF5801FF7D5994218BF704708BF904202
:1070700070474FF4001C1CEB430F38BF1CEB410F53
:1070800001D2994270470FB40CBC03BCFFF7C1BEDC
:1070900091EA030F10B581F000413FF5C1AB83F0D9
:1070A000004300F009B8000010B591EA030F48BF93
:1070B00083F000433FF5B4AB841A71EB030C07D2A5
:1070C00012198CF0004C43EB0C03001B61EB0C011C
:1070D000DFF8A4E14FEA1154A4EB135C1EEA430F5E
:1070E00018BF9EEA445F00F0B08023EA6E0352426C
:1070F00021EA0451C3EB6E0338BF5B1EDCF1200EA6
:1071000025D322FA0CFE10EB0E0043FA0CFE41EBE5
:107110000E01CCF1200E03FA0EFE10EB0E0051F121
:107120000001CCF1200E29D412FA0EF201EB045129
:10713000BDE8104058BF7047401C1CBFB2F1004F63
:10714000704700280CBF491C20F00100704712EB6B
:10715000020E43EB030218BF4FF0010E4EEA42024B
:10716000ACF1200CDCF11E0E54D943FA0CFE10EBEE
:107170000E0051F1FF31CCF11E0ED5D50EF1010EEE
:1071800012FA0EFE404141EB010101EB445C5FEA63
:107190005C5C10D910EBDE7001EB045138BFBEF11E
:1071A000004FBDE8104018BF704700280CBF491CB5
:1071B00020F00100704730D24FEAD42C11F50011B5
:1071C00024F400641BD0B1FA81F20B3AA41AA41E75
:1071D000D2F12003914030FA03F31943904001EBC0
:1071E000CC71002C01EB0451BDE81040A8BF7047E2
:1071F00001F1C0414FF0000001F000417047B0FACA
:1072000080F310FA03F100D110BDE41A173C4805D1
:10721000C90AE4E701EB045110BD491001EB045128
:10722000BDE810404FEA300002E04FF00001704727
:107230004A0008BF0042F8D0B2F5001F28BF7047CF
:1072400001F000414FF0000070479EEA445F07D014
:1072500011EA5E0FBDE8104004BF00210020704716
:10726000BDE8104070B5FFF789FE00BF40DFF63E75
:1072700083F00041104670470000E0FF00C18140EC
:1072800001C0804101C0804100C1814001C08041F6
:1072900000C1814000C1814001C0804101C08041E6
:1072A00000C1814000C1814001C0804100C18140D6
:1072B00001C0804101C0804100C1814001C08041C6
:1072C00000C1814000C1814001C0804100C18140B6
:1072D00001C0804101C0804100C1814000C18140A6
:1072E00001C0804101C0804100C1814001C0804196
:1072F00000C1814000C1814001C0804101C0804186
:1073000000C1814000C1814001C0804100C1814075
:1073100001C0804101C0804100C1814000C1814065
:1073200001C0804101C0804100C1814001C0804155
:1073300000C1814000C1814001C0804100C1814045
:1073400001C0804101C0804100C1814001C0804135
:1073500000C1814000C1814001C0804101C0804125
:1073600000C1814000C1814001C0804100C1814015
:1073700001C0804101C0804100C1814000C0C10105
:10738000C30302C2C60607C705C5C404CC0C0DCD95
:107390000FCFCE0E0ACACB0BC90908C8D81819D905
:1073A0001BDBDA1A1EDEDF1FDD1D1CDC14D4D51535
:1073B000D71716D6D21213D311D1D010F03031F125
:1073C00033F3F23236F6F737F53534F43CFCFD3D55
:1073D000FF3F3EFEFA3A3BFB39F9F83828E8E92945
:1073E000EB2B2AEAEE2E2FEF2DEDEC2CE42425E5F5
:1073F00027E7E62622E2E323E12120E0A06061A165
:1074000063A3A26266A6A767A56564A46CACAD6D14
:10741000AF6F6EAEAA6A6BAB69A9A86878B8B97984
:10742000BB7B7ABABE7E7FBF7DBDBC7CB47475B5B4
:1074300077B7B67672B2B373B17170B050909151A4
:107440009353529296565797559594549C5C5D9DD4
:107450005F9F9E5E5A9A9B5B9959589888484989C4
:107460004B8B8A4A4E8E8F4F8D4D4C8C4484854574
:107470008747468682424383418180405500000011
:107480000000000055000000000000005500000052
:1074900000000000B474000800000020A0010000FB
:1074A0006C01000840750008A001002000250000C4
:1074B000C80100080118F214B2010223FF092224B6
:1074C000B9602C02030404180A060708090204061E
:1074D000080171320A2904297C135D5739143202DC
:1074E000690413394C2A081D4BE8030432054B99F3
:1074F0004B283264290432045AE514322829043214
:107500000C4BDD4E14693C32061A951429504BD0B1
:107510000704190311CB814D142A0D64CA51783226
:10752000094BF554142984290429B8DA99A03208A2
:10753000CB655214320BCB7553142A0E44295031AB
:0400000508000131BD
:00000001FF
